:060000000CEF00F000000F
:10000800D8CFFFF5E0CF0FF0FACFFEF5D1EF14F01F
:1000180000EE10F012EE6DF0E4EC3EF005EE71F03B
:1000280015EEE2F0E4EC3EF000EEC6F011EE00F062
:10003800640EF66E000EF76E000EF86EDBEC3EF006
:1000480005EE6FF015EE71F0040EF66E000EF76E09
:10005800000EF86EDBEC3EF029EF15F019060A06E3
:1000680005060F06000614061E0690062A06430615
:10007800CF0665067B06B406A8064D063A06F807BD
:10008800B1071F08D107800A690A4D0A920A030BB3
:10009800E20AAA0A300AFFFF0101006F3F0EC716E5
:1000A800C66AC56AC686C75094869488C68A0051AF
:1000B800C86E1200FFFFF0D7AF01FFFFAFC1B1F16B
:1000C800B0C1B2F10101B36FC5CF00F01F0E001629
:1000D80000C002F0036A000EC7B4010E02120350FA
:1000E8000210D8A4F1D7C580C5B0FED7A1B632D0CA
:1000F8000101B35174D90009D8A42CD0C5CF00F0A0
:100108001F0E001600C002F0036A000EC7B4010EED
:10011800021203500210D8A4F1D7C5BC30D0010197
:10012800B2515DD90009D8A415D0C5CF00F01F0E73
:10013800001600C002F0036A000EC7B4010E0212D6
:1001480003500210D8A4F1D70101B15148D90009D0
:10015800D8B402D0010E14D0C5CF00F01F0E00167F
:1001680000C002F0036A000EC7B4010E0212035069
:100178000210D8A4F1D7C5BC02D0000E01D0020EDF
:100188001200FFFF9BD78101FFFF0101846F81C12E
:10019800AFF182C1B0F191DF0101836F8351D8A41F
:1001A80006D0C0D80101836F8351D8B402D08351DF
:1001B80030D0C5CF00F01F0E001600C002F0036A51
:1001C800000EC7B4010E021203500210D8A4F1D7D2
:1001D800C580C5B0FED7A1B606D001018429FFD8D5
:1001E8000009D8B402D0010E14D0C5CF00F01F0EFC
:1001F800001600C002F0036A000EC7B4010E021216
:1002080003500210D8A4F1D7C5BC02D0000E01D00B
:10021800020E1200FFFFB9D7FFFF0101AE6FC5CF75
:1002280000F01F0E001600C002F0036A000EC7B4EB
:10023800010E021203500210D8A4F1D70101AE51E9
:10024800CED80009D8B402D0010E14D0C5CF00F022
:100258001F0E001600C002F0036A000EC7B4010E9C
:10026800021203500210D8A4F1D7C5BC02D0000E68
:1002780001D0020E1200FFFFD0D7FFFFC5CF00F05C
:100288001F0E001600C002F0036A000EC7B4010E6C
:10029800021203500210D8A4F1D7C584C5A4000CDB
:1002A800FDD7FFFFEBD7FFFFA8D8C5B6FED7C59A85
:1002B800C588C5B8FED7C9501200FFFFF5D7FFFFA4
:1002C8009CD8C5B6FED7C58AC588C5B8FED7C5842B
:1002D800C5A4000CFDD7FFFFF3D77A01FFFF01018A
:1002E800806F7AC181F17BC182F14EDF01017F6F9E
:1002F8007F51D8B40BD012D0D6DF7CC1E9FF7DC1C5
:10030800EAFFEF6E01017C2B000E7D2301017E07C1
:100318007E29D8A4F1D7D3DF01017F6F7F51120066
:10032800FFFFDDD7FFFFC5CF00F01F0E001600C08E
:1003380002F0036A000EC7B4010E02120350021045
:10034800D8A4F1D7C584C5B4FED7A1A602D0010EA2
:1003580001D0000E1200FFFFE6D7FFFF0101AF6FCB
:10036800C5CF00F01F0E001600C002F0036A000E91
:10037800C7B4010E021203500210D8A4F1D7C580E9
:10038800C5B0FED7A1B624D00101AF5128D80009C5
:10039800D8A41ED0C5CF00F01F0E001600C002F072
:1003A800036A000EC7B4010E021203500210D8A44B
:1003B800F1D7A1B60DD0C5BC03D00101AE6B03D0F7
:1003C800040E0101AE6FC584C5B4FED7A1A602D044
:1003D800010E02D00101AE511200FFFFBFD7FFFF8F
:1003E800C96E0101B46FC6AE02D0FF0E03D0C7B00C
:0803F800FED7000E1200FFFF0A
:10040000F3D7FFFFC586C7A0FED7C9501200FFFF74
:10041000F9D7FFFF01D0FFFFF00E83160F0E9512E4
:10042000959A9598929A839A8398809ACAEC1AF032
:10043000F00E951683168382808AD6EC1AF0809A85
:10044000D0EC1AF0F00E83168382808AD6EC1AF074
:10045000809AD6EC1AF0F00E83168382808AD6EC4E
:100460001AF0809A0F0E9512280E0BD8280E09D874
:10047000080E07D80C0E05D8010E03D8130E01D8AC
:10048000800EFFFF01012B6F25D80009D8A4FCD7EF
:10049000959A9598F00E9516831601012B390F0B3E
:1004A0008312839A8398D6EC1AF0808AD6EC1AF0DD
:1004B000809AF00E831601012B510F0B8312D6EC9C
:1004C0001AF0808AD6EC1AF0809A0F0E951212005C
:1004D000FFFFD8D7FFFF838A8398959A9598D6EC2B
:1004E0001AF0808AD6EC1AF083A60AD0809AD6EC4D
:1004F0001AF0808AD6EC1AF0809A839A010E09D0FD
:10050000809AD6EC1AF0808AD6EC1AF0809A839AF8
:10051000000E1200FFFFDFD72B01FFFF2BC1E9FF09
:100520002CC1EAFFEF5001012D6F2D51D8B406D038
:1005300028D801012B2B000E2C23F0D71200FFFF2F
:10054000EDD72B01FFFF2BC1F6FF2CC1F7FF050EE6
:10055000F76404D00800FFFFF55005D0F6CFE9FF9F
:10056000F7CFEAFFEF5001012D6F2D51D8B406D01F
:1005700008D801012B2B000E2C23E5D71200FFFF1A
:10058000E2D7FFFF01012E6FA5DF0009D8A4FCD739
:10059000959A9598F00E9516831601012E390F0B3A
:1005A00083128388839AD6EC1AF0808AD6EC1AF0EC
:1005B000809AF00E831601012E510F0B8312D6EC98
:1005C0001AF0808AD6EC1AF0809A0F0E951212005B
:1005D000FFFFD8D7FFFFD96E390ED96401D006D0FE
:1005E000300ED96001D002D0D88001D0D89012004E
:1005F000FFFFF1D7FFFFEECFE6FFE82EFBD7000CA1
:10060000504F5254005155495400504153530053D8
:10061000544F520041424F5200555345520032321E
:10062000302052656164790D0A00323330204C6FFE
:100630006767656420696E0D0A00323030206F6B89
:100640000D0A00323231204279650D0A003232360D
:10065000205472616E7366657220436F6D706C65B5
:1006600074650D0A00353032204E6F7420696D704C
:100670006C656D656E7465640D0A00353330204C11
:100680006F67696E2072657175697265640D0A0025
:100690003333312050617373776F726420726571E8
:1006A00075697265640D0A0031323520446F6E65DC
:1006B0002E0D0A00313530205472616E73666572FA
:1006C00072696E6720646174612E2E2E0D0A0035EA
:1006D0003030200D0A005458540048544D0047490A
:1006E0004600434749004A504700434C41005741A8
:1006F0005600746578742F706C61696E000000009C
:10070000000000000000746578742F68746D6C0040
:1007100000000000000000000000696D6167652FA7
:1007200067696600000000000000000000007465BA
:1007300078742F68746D6C000000000000000000E9
:100740000000696D6167652F6A70656700000000D1
:100750000000000000006170706C69636174696F73
:100760006E2F6A6176612D766D00617564696F2FF9
:10077000782D776176650000000000000000485485
:1007800054502F312E3020323030204F4B0D0A4341
:100790006F6E74656E742D747970653A20000D0A61
:1007A0000D0A0047455400494E4445582E48544DC3
:1007B00000485454502F312E3020323030204F4BCF
:1007C0000D0A436F6E74656E742D747970653A20EE
:1007D00000485454502F312E3020353033200D0A2C
:1007E0000D0A5365727669636520556E617661699D
:1007F0006C61626C650D0A00485454502F312E30E4
:1008000020343034204E6F7420666F756E640D0A8C
:100810000D0A4E6F7420666F756E642E0D0A000D02
:100820000A0D0A004D434850537461636B207632C1
:100830002E323000444843502F476C65616E696E1C
:10084000672E2E2E00426F6172642053657475709E
:100850002E2E2E002020202020202020202020208E
:100860002020202000434F4D4D414E44532E4347FE
:100870004900494E4445582E48544D006674700056
:100880006D6963726F63686970000D0A0D0A0D4D22
:10089000434850537461636B2044656D6F20417011
:1008A000706C69636174696F6E2076312E31202817
:1008B0004D434850537461636B2076322E32302C96
:1008C000204A756E2032342032303033290D0A0D23
:1008D0000A09313A204368616E676520426F617290
:1008E000642073657269616C206E756D6265722E2D
:1008F0000D0A09323A204368616E676520646566B7
:1009000061756C7420495020616464726573732E44
:100910000D0A09333A204368616E67652064656695
:1009200061756C74206761746577617920616464B6
:10093000726573732E0D0A09343A204368616E673D
:10094000652064656661756C74207375626E65748C
:10095000206D61736B2E0D0A09353A20456E616278
:100960006C652044484350202620495020476C6540
:10097000616E696E672E0D0A09363A20446973610B
:10098000626C652044484350202620495020476C23
:1009900065616E696E672E0D0A09373A20446F77DC
:1009A0006E6C6F6164204D50465320696D616765C0
:1009B0002E0D0A09383A205361766520262051759C
:1009C00069742E0D0A0D0A456E7465722061206DE2
:1009D000656E752063686F6963652028312D38293D
:1009E0003A20000D0A496E76616C696420696E7068
:1009F0007574207265636569766564202D20496E83
:100A00007075742069676E6F7265642E0D0A50727E
:100A100065737320616E79206B657920746F206334
:100A20006F6E74696E75652E2E2E0D0A0025750089
:100A30000D0A4E6F772072756E6E696E6720617059
:100A4000706C69636174696F6E2E2E2E000D0A44FE
:100A5000656661756C7420476174657761792041C2
:100A60006464726573732028000D0A4465666175BD
:100A70006C742049502041646472657373202800AF
:100A80000D0A53657269616C204E756D6265722046
:100A900028000D0A44656661756C74205375626E9A
:100AA0006574204D61736B2028000D0A52656164E6
:100AB0007920746F20646F776E6C6F6164204D5085
:100AC000465320696D616765202D20557365205858
:100AD0006D6F64656D2070726F746F636F6C2E0D37
:100AE0000A000D0A44484350202620495020476CF4
:100AF00065616E696E672064697361626C65642EFE
:100B00000D0A000D0A444843502026204950204732
:100B10006C65616E696E6720656E61626C65642EDE
:040B20000D0A0000BA
:100B2400FFFF60D0D96A00D0D950260D2E0EF324D1
:100B3400E16E000EF420E26E000EE76E00EE25F08A
:100B4400E150E926E250EA22FE0EEF1600EE25F00F
:100B5400E150E926E250EA22EF50FD0B0209EF6E64
:100B640000EE25F0E150E926E250EA22EF50FB0BBB
:100B74000409EF6E00EE25F0E150E926E250EA2286
:100B8400EF0EEF1600EE25F0E150E926E250EA22DE
:100B9400F70EEF1600EE0FF0E150E926E250EA22DC
:100BA400FF0EEF6E00EE21F0E150E926E250EA225A
:100BB400700EEE6E170EEE6E000EEE6E000EED6E03
:100BC400010ED926030ED96401D001D0ADD700019E
:100BD400000E286F040E296F2A6B2B6B2C6B2D6B68
:100BE4001200FFFF9FD70101FFFF64D0D96A00D034
:0C0BF400D950260D2E0EF324E16E000EE9
:100C0000F420E26EE750D8A401D001D04AD0010E02
:100C1000E76E00EE0BF0E150E926E250EA2201C156
:100C2000EEFF02C1EDFF00EE0DF0E150E926E250CB
:100C3000EA22000EEE6E000EED6E00EE07F0E150BF
:100C4000E926E250EA22000EEE6E000EEE6E000E75
:100C5000EE6E000EED6E00EE25F0E150E926E2505A
:100C6000EA22EF50FE0B0109EF6E00EE25F0E15095
:100C7000E926E250EA22F70EEF1600EE0FF0E150FF
:100C8000E926E250EA22FF0EEF6E00EE25F0E15079
:100C9000E926E250EA22EF50FD0B0209EF6ED9502F
:100CA00009D0010ED926030ED96401D001D0A2D7F4
:100CB000FE0E00D01200FFFF9BD70801FFFFE2D01D
:100CC000D96A01010C6B00D001010C51260D2E0ECA
:100CD000F324E16E000EF420E26EE750D8A401D0B8
:100CE00001D003D0010ED96E08D0010E01010C27EE
:100CF000030E0C6501D001D0E7D7D950D8A401D09C
:100D000001D002D0FE0EBCD00001010E2827000E3B
:100D1000292300EE0BF0E150E926E250EA2228C038
:100D2000EEFF29C0EDFF130E295D890ED8B4285DB2
:100D3000D8A001D001D004D0000E286F040E296F76
:100D400000EE25F0E150E926E250EA22FE0EEF1611
:100D500000EE0DF0E150E926E250EA220AC1EEFF72
:100D60000BC1EDFF00012A2B000E2B232C232D237A
:100D700000EE14F0E150E926E250EA222AC0EEFF2C
:100D80002BC0EEFF2CC0EEFF2DC0EEFF00EE18F0E2
:100D9000E150E926E250EA22000EEE6E000EEE6E01
:100DA000000EEE6E000EED6E010EE1240101466FA5
:100DB000000EE220476FE1CF0DF1E2CF0EF108C146
:100DC00048F109C149F10A0E4A6F4B6BE5EC3DF061
:100DD0000DC1D9FF0EC1DAFF010ED9240101726FD6
:100DE000000EDA20736F00EE0BF0D950E926DA50CE
:100DF000EA22EECF74F1EDCF75F100EE0DF0D9508F
:100E0000E926DA50EA22EECF76F1EDCF77F100EE67
:100E100014F0D950E926DA50EA22EECF78F1EECF7D
:100E200079F1EECF7AF1EECF7BF100EE18F0D950E8
:100E3000E926DA50EA22EECF7CF1EECF7DF1EECF5B
:100E40007EF1EECF7FF1020E806F8169826B836B42
:100E5000E9EC0CF00DC1E1FF0EC1E2FF030EE76EFD
:100E600000EE14F0E150E926E250EA22EE2A000EEC
:100E7000EE22EE22ED22ED52ED5201010C5100D096
:100E80001200FFFF1DD7FFFF11D0D96ED950260DDC
:100E90002E0EF324E96E000EF420EA6EEF50040AE1
:100EA000000ED8B4010E00D01200FFFFEED7FFFFF6
:100EB00078D0E96EE950260D2E0EF324D96E000E7F
:100EC000F420DA6EE9500101666FD9CF67F1DACF0D
:100ED00068F1DF50040AD8B401D001D007D067C14F
:100EE00069F168C16AF1F2EC0FF059D00101665165
:100EF000CED967C1E1FF68C1E2FF010EE124010123
:100F0000726F000EE220736F00EE0BF0E150E926E5
:100F1000E250EA22EECF74F1EDCF75F100EE0DF064
:100F2000E150E926E250EA22EECF76F1EDCF77F1FB
:100F300000EE14F0E150E926E250EA22EECF78F11B
:100F4000EECF79F1EECF7AF1EECF7BF100EE18F033
:100F5000E150E926E250EA22EECF7CF1EECF7DF1BE
:100F6000EECF7EF1EECF7FF1110E806F8169826B43
:100F7000836BE9EC0CF067C1E1FF68C1E2FF00EEB2
:100F800014F0E150E926E250EA22EE2A000EEE22A9
:100F9000EE22ED22ED52ED52050EE76E00D012006A
:100FA000FFFF87D7FFFFC8D0D96ED950260D2E0E70
:100FB000F324E16E000EF420E26E00EE0FF0E1503B
:100FC000E926E250EA22EF50006E0028D8A401D0B2
:100FD00001D002D0000EAED000EE25F0E150E9269F
:100FE000E250EA22EF50006E00B201D001D002D0F0
:100FF000000EA0D0010EE1240101726F000EE2206C
:10100000736F00EE0BF0E150E926E250EA22EECFDA
:1010100074F1EDCF75F100EE0DF0E150E926E250EC
:10102000EA22EECF76F1EDCF77F100EE14F0E15049
:10103000E926E250EA22EECF78F1EECF79F1EECF59
:101040007AF1EECF7BF100EE18F0E150E926E250A4
:10105000EA22EECF7CF1EECF7DF1EECF7EF1EECF46
:101060007FF1100E806F00EE0FF0E150E926E250A4
:10107000EA22EF50816F00EE10F0E150E926E250D5
:10108000EA22EECF82F1EDCF83F1E1CF70F1E2CF32
:1010900071F1E9EC0CF070C1E1FF71C1E2FF00EE0B
:1010A00010F0E150E926E250EA22EECF00F0EDCF59
:1010B00001F000EE14F0E150E926E250EA2200507F
:1010C000EE260150EE22000EEE22ED22ED52ED5200
:1010D00000EE25F0E150E926E250EA22FD0EEF167F
:1010E00000EE25F0E150E926E250EA22EF0EEF167D
:1010F000010100EE0FF07051E9267151EA22EF5024
:101100002CEC27F070C1E1FF71C1E2FF00EE0FF09F
:10111000E150E926E250EA22FF0EEF6E00EE25F0E4
:10112000E150E926E250EA22EF50FD0B0209EF6E92
:10113000010E00D01200FFFF37D7FFFF20D0D96E7D
:10114000D950260D3D0EF324E96E000EF420EA6E10
:10115000EF50006E0028D8A401D001D003D044EC99
:1011600026F00BD0D950260D530EF324E96E000E55
:10117000F420EA6EEF30010B00D01200FFFFDFD742
:101180006A01FFFF83D0D96ED950260D2E0EF324AD
:1011900001016E6F000EF4206F6FD9506B6F00EE7F
:1011A0000FF06E51E9266F51EA22EF50006E0028D1
:1011B000D8A401D001D028D000EE0FF06E51E9265E
:1011C0006F51EA22A9C5EFFF00EE0FF06E51E9263C
:1011D0006F51EA22EF501CEC27F0010100EE10F0F5
:1011E0006E51E9266F51EA22000EEE6E000EED6E92
:1011F000280EAA6FAB6B00EE0FF06E51E9266F510F
:10120000EA22EF5055EC29F0010100EE10F06E518A
:10121000E9266F51EA22EECF6CF1EDCF6DF1030EAE
:101220006D5DCA0ED8B46C5DD8A001D001D002D0DB
:10123000000E2AD0010100EE25F06E51E9266F5113
:10124000EA22EF50EF0B1009EF6E6A5150EC26F0D6
:10125000010E01016C27000E6D2300EE10F06E519F
:10126000E9266F51EA226CC1EEFF6DC1EDFF030E5E
:101270006D5DCA0ED8B46C5DD8A001D001D002D08B
:101280006B5190DE010E00D01200FFFF7CD7FFFFF4
:101290002AD0D96ED950260D2E0EF324E16E000E01
:1012A000F420E26EE1CF69F1E2CF6AF100EE25F0C1
:1012B000E150E926E250EA22EF50006E00B601D07C
:1012C00001D002D0000E0DD03EEC27F0010100EE5F
:1012D00025F06951E9266A51EA22F70EEF16010E50
:1012E00000D01200FFFFD5D70001FFFF4FD0D96E0D
:1012F000D950260D2E0EF324E16E000EF420E26E7E
:1013000000EE25F0E150E926E250EA22EF50006EAF
:1013100000A601D001D035D0E1CF00F1E2CF01F13C
:1013200000EE25F0E150E926E250EA22EF50006E8F
:1013300000A401D001D00FD0280E01016A6F6B6BA1
:1013400041EC29F0010100EE25F00051E9260151A0
:10135000EA22FB0EEF16010100EE25F00051E9260E
:101360000151EA22EF50EF0B1009EF6E00C140F17E
:1013700001C141F102C142F103C143F1DEEC26F0AB
:1013800003D0006A016A00D01200FFFFB0D76601E7
:10139000FFFF65D0D96ED950260D2E0EF324E16ED5
:1013A000000EF420E26E00EE25F0E150E926E25056
:1013B000EA22EF50006E00A601D001D04CD0E1CF60
:1013C00068F1E2CF69F100EE25F0E150E926E25044
:1013D000EA22EF50006E00A401D001D00FD0280EF9
:1013E00001016A6F6B6B41EC29F0010100EE25F001
:1013F0006851E9266951EA22FB0EEF16010100EE61
:1014000012F06851E9266951EA22EE50ED10D8A495
:1014100001D001D00DD03EEC27F0010100EE25F007
:101420006851E9266951EA22F70EEF16000E15D031
:10143000010100EE12F06851E9266951EA22EE0638
:10144000000EED5AC7EC26F066C1E9FF67C1EAFF5E
:10145000EF6E010E02D0000E00D01200FFFF9AD7EF
:10146000FFFF11D0D96ED950260D530EF324E96E2B
:10147000000EF420EA6EEF30006E00320030010BF7
:1014800000D01200FFFFEED7FFFF89D10101076BEB
:10149000066B00D001010651260D2E0EF324E16EDD
:1014A000000EF420E26E00EE25F0E150E926E25055
:1014B000EA22EF50006E00A601D00BD000EE25F01E
:1014C000E150E926E250EA22EF50006E00A802D077
:1014D00000D002D000D001D058D1E1CF08F1E2CF46
:1014E00009F1E750D8A401D013D0E750006E0004F2
:1014F000D8A40DD000D000EE25F0E150E926E2504E
:10150000EA22EF50006E00A002D000D001D001D03E
:1015100002D000D001D039D15DEC3EF000C00AF11C
:1015200001C00BF102C00CF103C00DF108C1E1FFD5
:1015300009C1E2FF00EE1DF0E150E926E250EA2287
:101540000101EE500A5D006EEE500B59016EEE5037
:101550000C59026EED500D59036EED52ED5200EE36
:1015600021F0E150E926E250EA22EE52EE52EE522C
:101570000350ED5C08E10250ED5C05E10150ED5CCB
:1015800002E10050EF5CD8A001D001D001D0FDD025
:1015900044EC26F00009D8A401D001D001D0FDD040
:1015A0005DEC3EF0010100EE1DF00851E926095105
:1015B000EA2200C0EEFF01C0EEFF02C0EEFF03C052
:1015C000EEFF08C1E1FF09C1E2FF00EE21F0E150AA
:1015D000E926E250EA22EE2A000EEE22EE22ED2269
:1015E000ED52ED5200EE1CF0E150E926E250EA2205
:1015F000EF2A55D0020E0101076F61D000EE1CF0FA
:10160000E150E926E250EA22EF50006E030E005C42
:10161000D8B001D001D004D0120E0101076F06D05E
:10162000E1CF69F1E2CF6AF1F2EC0FF048D0110E90
:101630000101076F050EE76E42D000EE1CF0E1508D
:10164000E926E250EA22EF50006E040E005CD8A0BA
:1016500001D001D007D0E1CF69F1E2CF6AF1F2EC1D
:101660000FF003D0010E0101076F29D000EE1CF02E
:10167000E150E926E250EA22EF50006E040E005CD1
:10168000D8A001D001D007D0E1CF69F1E2CF6AF153
:10169000F2EC0FF003D0100E0101076F10D0E750ED
:1016A000020AACE0010AA6E0070AC1E0010AC5E0AF
:1016B000030ADCE0010ADAE00D0ABFE000D0010114
:1016C0000751D8B401D001D060D008C1E1FF09C1F1
:1016D000E2FF0751100AD8B401D001D011D000EEBA
:1016E00014F0E150E926E250EA22C9EC3EF000C0D5
:1016F00004F001C005F002C006F003C007F00ED0F0
:1017000000EE14F0E150E926E250EA22EECF04F0B8
:10171000EECF05F0EECF06F0EECF07F0010EE1249C
:101720000101726F000EE220736F00EE0BF0E150CA
:10173000E926E250EA22EECF74F1EDCF75F100EE2A
:101740000DF0E150E926E250EA22EECF76F1EDCF3E
:1017500077F104C078F105C079F106C07AF107C0CD
:101760007BF100EE18F0E150E926E250EA22EECFDC
:101770007CF1EECF7DF1EECF7EF1EECF7FF1075120
:10178000806F8169826B836B24D9010E010106276A
:10179000030E066501D001D07DD61200FFFF76D67C
:1017A0000601FFFF14D10101190E406F010E416FB8
:1017B000140E426F436BDEEC26F00101190EAA6F86
:1017C000010EAB6F5CDB010100EE06F00651E9266D
:1017D0000751EA22EECF0DF1EECF0EF1EECF0FF171
:1017E000EECF10F104C211F105C212F106C213F1DD
:1017F00007C214F1156B060E166F08C117F109C167
:1018000018F117C1C5F118C1C6F1D3EC39F000C009
:1018100017F101C018F101010D0EC36F010EC46F65
:101820000C0EC56FC66B34EC3AF0001C026E011C46
:10183000036E02C00BF103C00CF1240E01016A6FAC
:101840006B6B41EC29F001010B5150EC26F00101CA
:101850000C5150EC26F0140E01016A6F6B6B41ECD9
:1018600029F008C1AAF109C1ABF1CED900C00BF132
:1018700001C00CF101EE29F00101EE520C51ED18FE
:101880000BC1E8FFD8B4EF18D8B401D001D004D010
:101890003EEC27F0010E99D0010125390F0B006EA7
:1018A000D8900036D8900034EC0FD96ED95008C1CA
:1018B00000F009C101F0005E000E015AEC0E002498
:1018C000086FFF0E0120096F25390F0B006E00C055
:1018D00002F0036AD89002360336D89002360336F7
:1018E000140E02246A6F000E03206B6F41EC29F086
:1018F0000101190E2D6F010E2E6F06C12FF107C1C8
:1019000030F1D2D901010A6FFE0E0A6101D001D077
:101910000FD006C12DF107C12EF1190E2F6F010E48
:10192000306F08C131F109C132F10A51F0DB4BD0FF
:101930003EEC27F001010A29D8A401D001D043D000
:1019400008C100F009C101F0026A036A00502127B2
:1019500001502223025023230350242326A301D025
:1019600003D026A102D000D002D000D009D00101BE
:10197000010E2127000E2223000E2323000E242314
:1019800006C172F107C173F11BC174F11CC175F17D
:1019900019C176F11AC177F121C178F122C179F12B
:1019A00023C17AF124C17BF11DC17CF11EC17DF1FF
:1019B0001FC17EF120C17FF1040E0101806F81699A
:1019C000826B836B06D8010E00D01200FFFFEBD6AE
:1019D0007201FFFF17D100D044EC26F00009D8B403
:1019E00001D001D0F9D774C196F175C197F176C1D4
:1019F00098F177C199F178C19AF179C19BF17AC1D7
:101A00009CF17BC19DF17CC19EF17DC19FF17EC1A6
:101A1000A0F17FC1A1F101013F0EA317F00EA217A3
:101A20008051A36F59EC27F000C0A4F101C0A5F1CB
:101A300001EEA4F0EE52040EED5C000ED8B4EF5CA3
:101A4000D8A001D001D006D00101000EA46F040E71
:101A5000A56F15D001EEA4F0EE52000EED5C370E2E
:101A6000D8B4EF5CD8A001D001D006D00101CA0ED5
:101A7000A427FF0EA52303D00101A46BA56B0101D0
:101A8000A66BA76BA86BA96B960EAA6F010EAB6F26
:101A9000F6D9140E01018227000E832380A301D002
:101AA00001D010D0040E8227000E8323020E866F11
:101AB000040E876F040E886F896BA2510F0B6009AB
:101AC000A26F05D00101A2510F0B5009A26F04C2F1
:101AD0008AF105C28BF106C28CF107C28DF10101BA
:101AE00000EE06F07251E9267351EA22EECF8EF134
:101AF000EECF8FF1EECF90F1EECF91F1926B060E1B
:101B0000936F82C194F183C195F194C1C5F195C1E0
:101B1000C6F1D3EC39F000C094F101C095F1010198
:101B20008A0EC36F010EC46F0C0EC56FC66B34EC0A
:101B30003AF0001C026E011C036E02C0A6F103C045
:101B4000A7F1A6C184F1A7C185F101018129D8A41B
:101B500001D001D002D0A9C581F1140E0101AA6FF4
:101B6000AB6B815155EC29F072C1AAF173C1ABF195
:101B7000060E0101AC6F82C1ADF183C1AEF195ECEF
:101B800037F00101960ECB6F010ECC6F140ECD6FA6
:101B9000CE6B6BEC26F0010180A301D001D009D0FF
:101BA000860ECB6F010ECC6F040ECD6FCE6B6BEC3F
:101BB00026F0140E0101AA6FAB6B815155EC29F090
:101BC00082C1AAF183C1ABF11FD800C084F101C06A
:101BD00085F1240E0101AA6FAB6B815155EC29F000
:101BE0000101855150EC26F00101845150EC26F0A2
:101BF0000101AA6BAB6B815155EC29F0A9EC28F0DF
:101C00001200FFFFE8D6AA01FFFF4CD0010E010130
:101C1000AC6FAE6BAF6B29D0C7EC26F00101AD6F96
:101C2000AC51D8A401D001D00DD0AD51AE25AE6FCE
:101C3000AD51AE6101D001D004D0AF3F02D0010E52
:101C4000AE270DD00101AD51AF25AF6FAD51AF61E2
:101C500001D001D004D0AE3F02D0010EAF27010168
:101C6000AC51000ED8B4010EAC6F0101AA51006E48
:101C7000AB51016E010EAA5F000EAB5B015000106C
:101C8000D8A401D001D0C8D70101AF51FF0AAF6F6E
:101C9000AE51FF0AAE6FAEC100F0AFC101F000D08F
:101CA0001200FFFFB3D72D01FFFFE7D0FE0E0101A9
:101CB000316F016A00D00150260D2E0EF324D96E2B
:101CC000000EF420DA6EDF50D8B401D001D057D026
:101CD000010110EE02F02D51E1262E51E22200EE1C
:101CE0000BF0D950E926DA50EA22EE52E652E550DE
:101CF000ED18E7CFE8FFD8B4EF18D8A401D001D091
:101D00003ED0DF50006E0004D8A401D001D002D034
:101D10000150316F2DC1E9FF2EC1EAFF10EE0DF029
:101D2000D950E126DA50E222E652EE52ED50E518A3
:101D3000EFCFE8FFD8B4E718D8A41DD000D0010138
:101D400010EE06F02F51E1263051E22200EE07F0AE
:101D5000D950E926DA50EA22EE50E61808E1EE50B2
:101D6000E61805E1EE50E61802E1EE50E618D8A4B8
:101D700002D000D002D000D002D001507CD0010EA1
:101D80000126030E016401D001D095D70101315124
:101D9000260D2E0EF324E16E000EF420E26E31517A
:101DA000FE0AD8B408D000D0E750006E0004D8A4D2
:101DB00002D000D002D000D053D0010EE1240101A6
:101DC000466F000EE220476FE1CF32F1E2CF33F1F0
:101DD0002FC148F130C149F10A0E4A6F4B6BE5EC57
:101DE0003DF032C1D9FF33C1DAFF010110EE02F03C
:101DF0002D51E1262E51E22200EE0BF0D950E926BA
:101E0000DA50EA22E6CFEEFFE5CFEDFF2DC1E9FF84
:101E10002EC1EAFF10EE0DF0D950E126DA50E22291
:101E2000EECFE6FFEDCFE5FF00EE25F0D950E92635
:101E3000DA50EA22F70EEF1600EE0FF0D950E9263D
:101E4000DA50EA22FF0EEF6E00EE25F0D950E926B7
:101E5000DA50EA22EF50FD0B0209EF6E31510BD040
:101E600001013151FE0AD8A401D001D002D0FF0EE9
:101E700002D0FE0E00D01200FFFF18D7AA01FFFF0C
:101E8000AFD0AAC1E9FFABC1EAFFEECFC5F1EDCFFC
:101E9000C6F1D3EC39F0AAC1E9FFABC1EAFF00C03B
:101EA000EEFF01C0EDFF010100EE02F0AA51E926AC
:101EB000AB51EA22EECFC5F1EDCFC6F1D3EC39F04C
:101EC000010100EE02F0AA51E926AB51EA2200C05E
:101ED000EEFF01C0EDFF00EE04F0AA51E926AB5180
:101EE000EA22EECFACF1EECFADF1EECFAEF1EECF18
:101EF000AFF1E9EC39F0010100EE04F0AA51E92656
:101F0000AB51EA2200C0EEFF01C0EEFF02C0EEFFBF
:101F100003C0EEFF00EE08F0AA51E926AB51EA2219
:101F2000EECFACF1EECFADF1EECFAEF1EECFAFF143
:101F3000E9EC39F0010100EE08F0AA51E926AB51B5
:101F4000EA2200C0EEFF01C0EEFF02C0EEFF03C0B8
:101F5000EEFF00EE0EF0AA51E926AB51EA22EECFD9
:101F6000C5F1EDCFC6F1D3EC39F0010100EE0EF072
:101F7000AA51E926AB51EA2200C0EEFF01C0EDFFF5
:101F800000EE10F0AA51E926AB51EA22EECFC5F1DE
:101F9000EDCFC6F1D3EC39F0010100EE10F0AA51FB
:101FA000E926AB51EA2200C0EEFF01C0EDFF00EED2
:101FB00012F0AA51E926AB51EA22EECFC5F1EDCFDE
:101FC000C6F1D3EC39F0010100EE12F0AA51E92676
:101FD000AB51EA2200C0EEFF01C0EDFF1200FFFF8F
:101FE00050D76901FFFF91D0010100EE0FF0695158
:101FF000E9266A51EA22EF50006E0028D8B401D0D9
:1020000001D01FD000EE0FF06951E9266A51EA2293
:10201000EF502CEC27F069C1E1FF6AC1E2FF00EE4E
:102020000FF0E150E926E250EA22FF0EEF6E00EEDB
:1020300025F0E150E926E250EA22EF50FD0B0209BB
:10204000EF6E69C1E1FF6AC1E2FF00EE07F0E15007
:10205000E926E250EA22000EEE6E000EEE6E000E51
:10206000EE6E000EED6E00EE0DF0E150E926E2504E
:10207000EA22000EEE6E000EED6EE1CF69F1E2CFC6
:102080006AF100EE25F0E150E926E250EA22EF5035
:10209000006E00A601D001D002D03EEC27F069C14D
:1020A000E1FF6AC1E2FF00EE25F0E150E926E250CF
:1020B000EA22F70EEF1600EE21F0E150E926E25099
:1020C000EA22700EEE6E170EEE6E000EEE6E000E31
:1020D000ED6E00EE25F0E150E926E250EA22EF0E27
:1020E000EF1600EE25F0E150E926E250EA22EF502B
:1020F000006E00A001D001D003D0010EE76E02D027
:10210000000EE76E00D01200FFFF6ED72D01FFFF1B
:102110008BEF14F0D96E0101336BD950260D2E0EC2
:10212000F324E16E000EF420E26E00EE18F0E150B0
:10213000E926E250EA22EECF36F1EECF37F1EECFCC
:1021400038F1EECF39F100EE14F0E150E926E2501B
:10215000EA22EECF3AF1EECF3BF1EECF3CF1EECFFB
:102160003DF100EE04F02F51E9263051EA22EECF86
:1021700042F1EECF43F1EECF44F1EECF45F131C164
:1021800000F032C101F0026A036A00504227015098
:102190004323025044230350452300EE14F0E15042
:1021A000E926E250EA22EECF3EF1EECF3FF1EECF4C
:1021B00040F1EECF41F100EE1CF0E150E926E25093
:1021C000EA22000EEF6EE1CF34F1E2CF35F15DECA3
:1021D0003EF0010100EE1DF03451E9263551EA22AE
:1021E00000C0EEFF01C0EEFF02C0EEFF03C0EEFF35
:1021F00034C1D9FF35C1DAFF00EE21F0D950E9260C
:10220000DA50EA22700EEE6E170EEE6E000EEE6ED3
:10221000000EED6EDF50006E0004D8A401D001D096
:10222000ABD03EEC27F034C1D9FF35C1DAFF000155
:102230002A2B000E2B232C232D2300EE14F0D95033
:10224000E926DA50EA222AC0EEFF2BC0EEFF2CC0AE
:10225000EEFF2DC0EEFF0101010E4227000E4323C9
:10226000000E4423000E452300EE18F0D950E92655
:10227000DA50EA2242C1EEFF43C1EEFF44C1EEFF55
:1022800045C1EEFF00EE14F0D950E926DA50EA22FB
:10229000EECF3EF1EECF3FF1EECF40F1EECF41F188
:1022A00000EE14F0D950E926DA50EA22EE2A000EA8
:1022B000EE22EE22ED22ED52ED522FC1E1FF30C1B0
:1022C000E2FF00EE0DF0E150E926E250EA22EF5085
:1022D000006E00A201D001D027D0010ED924466F94
:1022E000000EDA20476F2DC148F12EC149F10A0EC8
:1022F0004A6F4B6BE5EC3DF034C1D9FF35C1DAFFD5
:102300002FC1E9FF30C1EAFF10EE0DF0D950E126F0
:10231000DA50E222EECFE6FFEDCFE5FF120E01012B
:10232000336F020EDF6E27D0040E0101336F42C1FE
:102330003EF143C13FF144C140F145C141F100EEDE
:1023400004F0E150E926E250EA22EECF42F1EECF6E
:1023500043F1EECF44F1EECF45F100EE07F0D95056
:10236000E926DA50EA22000EEE6E000EEE6E000E46
:10237000EE6E000EED6E9AD22FC1E1FF30C1E2FF8A
:1023800000EE0DF0E150E926E250EA22EF50006E37
:1023900000A401D001D008D03EEC27F034C169F18F
:1023A00035C16AF11FDEB5D200EE08F0E150E92632
:1023B000E250EA220101EE503E1908E1EE503F19C9
:1023C00005E1EE50401902E1EE504119D8A401D0C8
:1023D00001D06AD2DF50020AD8A401D001D064D063
:1023E00000EE0DF0E150E926E250EA22EF50006ED7
:1023F00000A801D001D055D000EE18F0D950E92640
:10240000DA50EA2242C1EEFF43C1EEFF44C1EEFFC3
:1024100045C1EEFF00EE1CF0D950E926DA50EA2261
:10242000000EEF6E5DEC3EF0010100EE1DF0345148
:10243000E9263551EA2200C0EEFF01C0EEFF02C0DE
:10244000EEFF03C0EEFF34C1E1FF35C1E2FF040E31
:10245000E76E32513111D8B401D001D01FD000EE57
:1024600025F0E150E926E250EA22EF50F70B080987
:10247000EF6E00EE12F0E150E926E250EA2231C19F
:10248000EEFF32C1EDFF00EE25F0E150E926E2500B
:10249000EA22EF50FB0B0409EF6E02D03EEC27F06E
:1024A00002D03EEC27F0FFD1DF50030AD8A401D0C0
:1024B00001D07BD000EE0DF0E150E926E250EA2297
:1024C000EF50006E00A201D001D06CD00101010ECE
:1024D0004227000E4323000E4423000E452300EE46
:1024E00018F0D950E926DA50EA2242C1EEFF43C182
:1024F000EEFF44C1EEFF45C1EEFF00EE0DF0E150EE
:10250000E926E250EA22EF50006E00A801D001D087
:1025100005D0100E336F040EDF6E1BD0120E0101BA
:10252000336F020EDF6E010E3E27000E3F23000EBA
:102530004023000E412300EE14F0D950E926DA5072
:10254000EA223EC1EEFF3FC1EEFF40C1EEFF41C1B6
:10255000EEFF010132513111D8B401D001D01FD0AA
:1025600000EE25F0D950E926DA50EA22EF50F70BB9
:102570000809EF6E00EE12F0D950E926DA50EA228F
:1025800031C1EEFF32C1EDFF00EE25F0D950E92652
:10259000DA50EA22EF50FB0B0409EF6E02D03EEC5A
:1025A00027F002D03EEC27F07ED110EE18F0D95083
:1025B000E126DA50E222010100EE04F02F51E92673
:1025C0003051EA22EE50E61808E1EE50E61805E137
:1025D000EE50E61802E1EE50E618D8B401D001D072
:1025E00003D03EEC27F095D100EE18F0D950E92643
:1025F000DA50EA2242C1EEFF43C1EEFF44C1EEFFD2
:1026000045C1EEFFDF50040AD8A401D001D0C9D0E3
:10261000010100EE0DF02F51E9263051EA22EF5072
:10262000006E00A801D001D02CD000EE0FF0D950E0
:10263000E926DA50EA22EF50006E0028D8B401D023
:1026400001D01FD000EE0FF03451E9263551EA22B7
:10265000EF502CEC27F034C1D9FF35C1DAFF00EE82
:102660000FF0D950E926DA50EA22FF0EEF6E00EEA5
:1026700025F0D950E926DA50EA22EF50FD0B020985
:10268000EF6E010100EE0DF02F51E9263051EA22E4
:10269000EF50006E00A001D001D02BD0110E336F8F
:1026A00000EE14F0D950E926DA50EA22C9EC3EF0E7
:1026B00000C03EF101C03FF102C040F103C041F152
:1026C00000EE18F0D950E926DA50EA22EE2A000E80
:1026D000EE22EE22ED22ED52ED52EECF42F1EECFA0
:1026E00043F1EECF44F1EDCF45F1ED52ED520A0E3C
:1026F000DF6E010132513111D8B401D001D04ED07A
:1027000000EE25F0D950E926DA50EA22EF50006EAB
:1027100000B601D001D021D000EE25F0D950E92635
:10272000DA50EA22EF50F70B0809EF6E00EE12F0D4
:10273000D950E926DA50EA2231C1EEFF32C1EDFF6D
:1027400000EE25F0D950E926DA50EA22EF50FB0BD3
:102750000409EF6E100E336F20D00101336B00EED1
:1027600014F0D950E926DA50EA223AC1EEFF3BC113
:10277000EEFF3CC1EEFF3DC1EEFF00EE18F0D95078
:10278000E926DA50EA2236C1EEFF37C1EEFF38C142
:10279000EEFF39C1EEFF3EEC27F002D03EEC27F011
:1027A00082D0DF500A0AD8A401D001D015D03EEC67
:1027B00027F0010100EE0DF02F51E9263051EA22F9
:1027C000EF50006E00A801D001D005D034C169F1EE
:1027D00035C16AF107DC67D0DF50050AD8A401D003
:1027E00001D046D03EEC27F02FC1E1FF30C1E2FF1F
:1027F00000EE0DF0E150E926E250EA22EF50006EC3
:1028000000A001D001D033D0100E0101336F34C1CC
:10281000D9FF35C1DAFF00EE18F0D950E926DA50B9
:10282000EA22EE2A000EEE22EE22ED22ED52ED52C9
:10283000EECF42F1EECF43F1EECF44F1EDCF45F1D3
:10284000ED52ED5200EE0DF0E150E926E250EA22A1
:10285000EF50006E00A801D001D007D0D9CF69F1A8
:10286000DACF6AF1F2EC0FF002D0060EDF6E1BD069
:10287000DF50060AD8A401D001D015D03EEC27F0D5
:10288000010100EE0DF02F51E9263051EA22EF5000
:10289000006E00A801D001D006D034C169F135C165
:1028A0006AF1F2EC0FF002D03EEC27F00101335157
:1028B000D8B401D001D02DD02DC172F12EC173F149
:1028C0002FC1E1FF30C1E2FF00EE02F0E150E92646
:1028D000E250EA22EECF74F1EDCF75F1E6CF76F15A
:1028E000E5CF77F13EC178F13FC179F140C17AF18E
:1028F00041C17BF142C17CF143C17DF144C17EF114
:1029000045C17FF13351806F8169826B836BE9EC44
:102910000CF01200FFFF8AEF10F0FFFF6BEC3EF0AF
:10292000E2C5F3FFE3C5F4FFE4C5F5FFE5C5F6FF37
:10293000E6C5F7FFE7C5F8FFE8C500F0E9C501F017
:10294000EAC502F0EBC503F0ECC504F0EDC505F0F7
:10295000EEC506F0EFC507F0F0C508F0F1C509F0C7
:10296000F2C50AF0F3C50BF0F4C50CF0F5C50DF097
:10297000F6C50EF0F7C5DAFFF8C5D9FFF9C5E2FFD5
:10298000FAC5E1FFFBC5EAFFFCC5E9FFFDC5E8FFAD
:10299000FACFFEF50FC0E0FFFFC5D8FF1000FFFF24
:1029A000BDD7FFFFE8CFFDF5E9CFFCF5EACFFBF59A
:1029B000E1CFFAF5E2CFF9F5D9CFF8F5DACFF7F5AF
:1029C0000EC0F6F50DC0F5F50CC0F4F50BC0F3F52F
:1029D0000AC0F2F509C0F1F508C0F0F507C0EFF53F
:1029E00006C0EEF505C0EDF504C0ECF503C0EBF54F
:1029F00002C0EAF501C0E9F500C0E8F5F8CFE7F557
:102A0000F7CFE6F5F6CFE5F5F5CFE4F5F4CFE3F54E
:102A1000F3CFE2F582D7FFFF0101AD6FACA2FED785
:102A20000101AD51AD6E1200FFFFF6D72B01FFFF84
:102A30002BC1E9FF2CC1EAFF01012B4B2C2BEF50DE
:102A40002D6F2D51D8B402D0E6DFF2D71200FFFF70
:102A5000EFD7FFFFAFDA50EC3EF014EC35F0CBDAF5
:102A600081BA0CD0C00E41EC02F00101450E2B6F73
:102A7000080E2C6FA2EC02F0FDEC19F048EC38F0D7
:102A800000EC20F085EC29F01CC200F000A00BD077
:102A9000C00E41EC02F00101340E2B6F080E2C6FBA
:102AA000A2EC02F006D0010EE8CFD1F5070EE8CF78
:102AB0006FF55DEC3EF000C2E8FF005C046E01C201
:102AC000E8FF0158056E02C2E8FF0258066E03C215
:102AD000E8FF0358076E000E075C08E1000E065C75
:102AE00005E1000E055C02E1320E045CD8A00BD0BB
:102AF0005DEC3EF000C000F201C001F202C002F243
:102B000003C003F2897859EC38F02BEC20F09DECEF
:102B100029F00ED972C5E8FF0501D119D8B4C9D77B
:102B20000101040E1E6F020E1F6F010E206F1AD8D6
:102B300072C5D1F51CC200F000A0BBD7CE0E41EC8F
:102B400002F00A0E0501D16106D0D1C5E8FF300FB1
:102B5000C1EC02F0AED7D1C5E8FF410FC1EC02F0E5
:102B6000A8D71E01FFFF01012051C00ED8B40AD022
:102B700041EC02F00101540E2B6F080E2C6FA2ECF9
:102B800002F0C00E41EC02F00101210E2D6F010E8A
:102B90002E6F2D0E2F6F0A0E306F1EC1E9FF1FC161
:102BA000EAFFEF50006E00C002F0036A02C029F194
:102BB00003C02AF1290EE8CF2BF1010EE8CF2CF14A
:102BC00077EC30F001012051D8B40AD0210E2B6FE0
:102BD000010E2C6F8DEC02F02E0EC1EC02F008D02D
:102BE0000101210E2B6F010E2C6F21DF2E0E13DF42
:102BF0000101210E2D6F010E2E6F2D0E2F6F0A0E6B
:102C0000306F00EE01F01E51E9261F51EA22EF500D
:102C1000006E00C002F0036A02C029F103C02AF16D
:102C2000290EE8CF2BF1010EE8CF2CF177EC30F034
:102C300001012051D8B40AD0210E2B6F010E2C6F48
:102C40008DEC02F02E0EC1EC02F008D00101210E35
:102C50002B6F010E2C6FEBDE2E0EDDDE0101210E3F
:102C60002D6F010E2E6F2D0E2F6F0A0E306F00EE9E
:102C700002F01E51E9261F51EA22EF50006E00C0FB
:102C800002F0036A02C029F103C02AF1290EE8CF3D
:102C90002BF1010EE8CF2CF177EC30F0010120513F
:102CA000D8B40AD0210E2B6F010E2C6F8DEC02F0E0
:102CB0002E0EC1EC02F008D00101210E2B6F010E87
:102CC0002C6FB5DE2E0EA7DE0101210E2D6F010E39
:102CD0002E6F2D0E2F6F0A0E306F00EE03F01E5177
:102CE000E9261F51EA22EF50006E00C002F0036A8D
:102CF00002C029F103C02AF1290EE8CF2BF1010E01
:102D0000E8CF2CF177EC30F001012051D8B407D096
:102D1000210E2B6F010E2C6F8DEC02F006D00101FD
:102D2000210E2B6F010E2C6F82DE1200FFFF1BD7CE
:102D3000FFFF810EC26E640E0101006F01010007EA
:102D40000029D8A4FBD7C284C2B4FED7C350010166
:102D5000006FC450016FD20E2D6F050E2E6F2D0E19
:102D60002F6F0A0E306F00C102F101C103F1020E94
:102D7000E8CF2BF1010EE8CF2CF177EC30F0840E88
:102D8000C16E890EC26E640E0101006F0101000761
:102D90000029D8A4FBD7C284C2B4FED7C350010116
:102DA000006FC450016FDA0E2D6F050E2E6F2D0EC1
:102DB0002F6F0A0E306F00C102F101C103F1020E44
:102DC000E8CF2BF1010EE8CF2CF177EC30F08E0E2E
:102DD000C16E1200FFFFADD76601FFFF66C1E9FFBC
:102DE00067C1EAFFEECF00F0EDCF01F000C0E9FFD0
:102DF00001C0EAFFEF50D00F0101696F2ED0010131
:102E000000EE02F06651E9266751EA22EECF00F0AB
:102E1000EDCF01F000C0E9FF01C0EAFFEF50D00F95
:102E20006A6F04D0897607D0897405D001016A5190
:102E3000F9E0010AF9E066C1E9FF67C1EAFFEECFF8
:102E400076F1EDCF77F10101650E786F080E796F9D
:102E50000D0E7A6FCFEC3AF015D001016951CFE039
:102E6000010AFAE066C1E9FF67C1EAFFEECF76F139
:102E7000EDCF77F1720E786F080E796F0A0E7A6FC8
:102E8000CFEC3AF01200FFFFA9D76A01FFFF010162
:102E90006E6F53D089B603D049D089A447D06CC196
:102EA000E9FF6DC1EAFF300E46D001016B516A1196
:102EB000D8A402D06A6B6B6B01016A5115EED2F097
:102EC000E126000EE2226CC1E9FF6DC1EAFFE7CF07
:102ED000EFFF6A5105EED2F0E926000EEA22EF502C
:102EE000D8A419D035D001016B516A11D8A402D0F1
:102EF0006A6B6B6B01016A5115EEDAF0E126000E88
:102F0000E2226CC1E9FF6DC1EAFFE7CFEFFF6A5132
:102F100005EEDAF0E1D701016A2B000E6B236AC1DE
:102F200000F06BC101F017D081AAB9D76CC1E9FFDD
:102F30006DC1EAFF310EEF6E0BD001016E51AAE0B8
:102F4000010AABE0030AB1E0010ACDE0070AECE0B8
:102F5000FF0E006801681200FFFF99D70701FFFF0D
:102F600007C176F108C177F101017C0E786F080E78
:102F7000796F030E7A6F7B6B49EC3DF001500010C6
:102F8000D8A414D009C176F10AC177F10101800EED
:102F9000786F080E796F090E7A6F7B6B49EC3DF004
:102FA00001500010D8A402D0010E01D0000E120072
:102FB000FFFFD6D7FFFF8E0EC16E030E926E809A72
:102FC00089848986F19E09EC02F0800E41EC02F0C2
:102FD0000101240E2B6F080E2C6FA2EC02F0200EC4
:102FE000AC6E900EAB6E0F0EAF6ED56AF28EF28C99
:102FF0001200FFFFE0D7FFFF0A0EE8CF04F2E8CF90
:1030000005F2050EE8CF06F20F0EE8CF07F2FF0E2D
:10301000E8CF0EF2E8CF0FF2E8CF10F20201116B09
:103020000A0EE8CF12F2E8CF13F2050EE8CF14F241
:103030000F0EE8CF15F2086B040EE8CF09F2A30ECD
:10304000E8CF0AF20B6B0C6B0D6B1C810101040EB7
:10305000016F020E026F816B826BA00EC8EC00F054
:1030600057EC01F00101006F63EC01F00101005128
:10307000550AD8A41BD0010E816F826BA00EC8EC3C
:1030800000F00101006B0CD057EC01F001C1E9FF29
:1030900002C1EAFFEF6E0101012B000E0223002B9B
:1030A000180E0065F1D763EC01F001D003D81200CF
:1030B000FFFFA2D7FFFF0101040E1F6F020E206F5A
:1030C000AF6BB06BA00E61EC00F0550E10EC01F090
:1030D00001011E6B0CD01FC1E9FF20C1EAFF0101F5
:1030E0001F4B202BEF5010EC01F001011E2B180E8E
:1030F0001E65F1D741EF01F0FFFFDDD71E01FFFF95
:1031000001011EC1F6FF1FC1F7FF1E2B000E1F237A
:10311000050EF76404D00800FFFFF55005D0F6CF88
:10312000E9FFF7CFEAFFEF50206F2051D8B403D06A
:10313000010171DCE5D71200FFFFE2D71E01FFFF9E
:103140000101226B9EAAFED7AE500101216F0D0A2C
:10315000D8B417D021510A0AD8B413D0222B1EC1DB
:10316000E9FF1FC1EAFF21C1EFFF1E2B000E1F2345
:103170001EC1E9FF1FC1EAFFEF6A20072029D8A47A
:10318000E1D7010122511200FFFFDAD71E01FFFF34
:103190001EC123F11FC124F10101256B1EC1E9FFEE
:1031A0001FC1EAFFEF500101226F2251D8B42FD086
:1031B0002E0AD8A41DD01EC1E9FF1FC1EAFFEF6A85
:1031C0001E2B000E1F2323C126F124C127F128EC5A
:1031D0003CF0010125512025E96E000E2121EA6E07
:1031E00000C0EFFF252B1EC123F11FC124F10AD01F
:1031F000300E0101226101D003D0390E226502D0C8
:10320000000E19D001011E2B000E1F23C7D723C1AA
:1032100026F124C127F128EC3CF00101255120259D
:10322000E96E000E2121EA6E00C0EFFF2551030A6E
:10323000000ED8B4010E1200FFFFAAD7FFFF9EAA0E
:10324000FED7AE500101016F300E016505D0390E79
:10325000016102D0015101D0390E1200FFFFEFD7FA
:10326000FFFF01011B6F0D0E0BEC15F00A0E0BECAE
:1032700015F001011B51020D8E0EF324E96E000EB4
:10328000F420EA6EEECF1EF1EDCF1FF138DF9FD0B4
:103290000101010E2D6F010E2E6F2D0E2F6F0A0EE4
:1032A000306F02EE16F0EECF1CF1EDCF1DF11C0ECB
:1032B000E8CF2BF1010EE8CF2CF177EC30F00101D3
:1032C000010E2B6F010E2C6F17EC15F0290E0BEC75
:1032D00015F03A0E0BEC15F0200E0BEC15F0010179
:1032E000010E1E6F010E1F6F140E206F28DF006E7F
:1032F00000C002F0036A03500210D8B447D0010E98
:10330000266F010E276F28EC3CF000C016F201C0BA
:1033100017F217C20CF216C20DF26CD00101040EA6
:10332000196F020E09D00101120E196F020E04D09E
:1033300001010E0E196F020E1A6F19C11EF11AC18A
:103340001FF10101206B0EDC290E0BEC15F03A0E7B
:103350000BEC15F0200E0BEC15F00101010E1E6FA9
:10336000010E1F6F140E206FEADE010E1E6F010E9C
:103370001F6F150E206F010E216F09DF006E00C058
:1033800002F0036A03500210D8A40AD00101E30E30
:103390001E6F090E1F6FB3DE9EAAFED7AE502AD055
:1033A00019C1E9FF1AC1EAFF15C1EEFF16C1EEFF10
:1033B00017C1EEFF18C1EEFF1DD002011C811AD00B
:1033C00002011C9117D030D815D074DE13D0010142
:1033D0001B51310A01E15CD7030AA0E0010AA3E016
:1033E000070AA6E0010AE9E0030AEAE0010AEBE0C5
:1033F0000F0AEBE01200FFFF34D7FFFF01018A0E36
:103400001E6F080E1F6F7BDE19DF0101006F390A86
:10341000D8B402D0005124DF01010051380AD8B4D9
:103420001200ECD7FFFFEAD7FFFF01011E6B226BF2
:1034300026EC36F000C020F101C021F15DEC3EF039
:1034400000C0A5F101C0A6F102C0A7F103C0A8F118
:103450006BEC3EF05DEC3EF000C0A9F101C0AAF1BA
:1034600002C0ABF103C0ACF10101A551A95D006E32
:10347000A651AA59016EA751AB59026EA851AC5979
:10348000036E000E035C08E1000E025C05E1000E15
:10349000015C02E1320E005CD8A00ED05DEC3EF083
:1034A00000C0A5F101C0A6F102C0A7F103C0A8F1B8
:1034B000150E0BEC15F089749EBA65D0C9D76BEC6C
:1034C0003EF09EAA60D08974AE5001011F6F1E515C
:1034D000010A1DE0030A21E0010A22E01F05D8A429
:1034E00003D0010E1E6F4FD001011F51040AD8A452
:1034F0000AD08984BFEC35F0060E0BEC15F0010EF6
:103500000101226F40D0150E0BEC15F03CD0060ED9
:103510000101246F236B020EE5D7030E0101E2D7F0
:103520000101235101EE25F0E926000EEA221FC118
:10353000EFFF232B800E236526D020C1ADF121C1E2
:10354000AEF132EC36F0060E0101246F1F6B0CD089
:1035500001011F5101EE25F0E926000EEA22EF508D
:1035600051EC36F001011F2B7F0E1F65F1D77BEC6C
:1035700036F000C020F101C021F1010124510BEC13
:1035800015F001011E6B01012251D8A4010C97D73F
:10359000FFFF4BD7FFFF0F0EACEF3EF0FFFFFBD757
:1035A000FFFF040EACEF3EF0FFFFFBD7FFFFF29EE4
:1035B000010E01012F6F01012F2FFDD7F28E120096
:1035C000FFFFF5D7FFFF93D179D1010107690869A2
:1035D00009690A690B690C690D690E690F6910693F
:1035E0000001206B216B226B236B440E0101116FD4
:1035F000126B070E136F010E146F430E156F166BCF
:103600002BEC2DF0E8CF73F55DEC3EF000C010F030
:1036100001C011F002C012F003C013F0010EE8CF98
:103620006FF55DEC3EF010C0E8FF005C046E11C069
:10363000E8FF0158056E12C0E8FF0258066E13C07D
:10364000E8FF0358076E000E075C08E1000E065CF9
:1036500005E1000E055C02E1140E045CD8A001D067
:1036600001D003D0020EE8CF6FF53FD10001205109
:10367000211122112311D8B401D001D004D0040E9D
:10368000E8CF6FF518D073C5D0F544EC26F00009EB
:10369000D8B401D001D00FD0010EF6DA5DEC3EF0C7
:1036A00000C010F001C011F002C012F003C013F00E
:1036B000030EE8CF6FF519D173C5E8FFBDEC2EF00E
:1036C0000009D8B401D001D00AD01ED9020AD8A46A
:1036D00001D001D003D0040EE8CF6FF524D05DEC0B
:1036E0003EF010C0E8FF005C046E11C0E8FF015816
:1036F000056E12C0E8FF0258066E13C0E8FF0358BB
:10370000076E000E075C08E1000E065C05E1000E86
:10371000055C02E1C80E045CD8A001D001D003D042
:10372000020EE8CF6FF5E1D073C5D0F544EC26F07A
:103730000009D8B401D001D00FD0030EA5DA5DEC9A
:103740003EF000C010F001C011F002C012F003C042
:1037500013F0050EE8CF6FF5C8D073C5E8FFBDECD8
:103760002EF00009D8B401D001D044D0CDD8010149
:10377000066F0651060AD8A401D001D004D0040E69
:10378000E8CF6FF536D001010651050AD8A401D063
:1037900001D02FD073C5E8FF9BEC2DF05DEC3EF01F
:1037A00000C010F001C011F002C012F003C013F00D
:1037B000060EE8CF6FF520C004F221C005F222C04A
:1037C00006F223C007F224C00EF225C00FF226C075
:1037D00010F227C011F21CC012F21DC013F21EC05D
:1037E00014F21FC015F2050170810501010E722748
:1037F0007CD024D05DEC3EF010C0E8FF005C046E8D
:1038000011C0E8FF0158056E12C0E8FF0258066EAD
:1038100013C0E8FF0358076E000E075C08E1000EB6
:10382000065C05E1000E055C02E1C80E045CD8A050
:1038300001D001D003D0020EE8CF6FF556D05DEC79
:103840003EF010C0E8FF005C046E11C0E8FF0158B4
:10385000056E12C0E8FF0258066E13C0E8FF035859
:10386000076E000E075C08E1000E065C05E1000E25
:10387000055C02E1640E045CD8A001D001D01DD02B
:103880000001FF0E1427FF0E1523FF0E1623FF0E57
:1038900017231451151116111711D8A401D001D0F6
:1038A00002D005016F6B5DEC3EF000C010F001C06E
:1038B00011F002C012F003C013F017D06FC5E8FF7B
:1038C000000A01E182D6010A01E1ABD6030A01E157
:1038D000CDD6010A01E1F0D6070A01E125D7010A98
:1038E00001E13BD7030AABE000D01200FFFF6CD62A
:1038F000FFFF09D0080EE8CF6FF573C5E8FF9BEC1A
:103900002DF01200FFFFF6D7FFFFBDD10101126BB2
:103910000001000E176F000E166F000E156F3C0EA3
:10392000146F0101140E196F010E1A6FD0EC2EF0F6
:1039300001011451020AD8A401D001D078D1136B2F
:103940000E0E136501D001D001D00FD00101140E6D
:10395000196F010E1A6FD0EC2EF0010E0101132722
:103960000E0E136501D001D0F1D70101200E196FA1
:10397000000E1A6FD0EC2EF00101210E196F000E0F
:103980001A6FD0EC2EF00101220E196F000E1A6F83
:10399000D0EC2EF00101230E196F000E1A6FD0EC3F
:1039A0002EF00101136BDB0E136501D001D001D0A5
:1039B0000FD00101140E196F010E1A6FD0EC2EF00A
:1039C000010E01011327DB0E136501D001D0F1D7E1
:1039D0000101116B0101140E196F010E1A6FD0EC69
:1039E0002EF00CD10101140E196F010E1A6FD0ECDC
:1039F0002EF001011405D8A401D001D007D0120E79
:103A0000196F010E1A6FD0EC2EF001D038D109D108
:103A10000101140E196F010E1A6FD0EC2EF0010186
:103A20001451040AD8A401D001D01CD0240E196F5F
:103A3000000E1A6FD0EC2EF00101250E196F000E4A
:103A40001A6FD0EC2EF00101260E196F000E1A6FBE
:103A5000D0EC2EF00101270E196F000E1A6FD0EC7A
:103A60002EF001D00CD1DDD00101140E196F010E22
:103A70001A6FD0EC2EF0030E0101146501D001D0B5
:103A80001CD01C0E196F000E1A6FD0EC2EF0010125
:103A90001D0E196F000E1A6FD0EC2EF001011E0ED4
:103AA000196F000E1A6FD0EC2EF001011F0E196F66
:103AB000000E1A6FD0EC2EF001D0E1D0FC0E010107
:103AC000142707D00101130E196F010E1A6FD0ECE5
:103AD0002EF0010114071429D8A401D001D0F2D787
:103AE000A0D00101140E196F010E1A6FD0EC2EF048
:103AF00001011451040AD8A401D001D01CD0180E21
:103B0000196F010E1A6FD0EC2EF00101170E196F0C
:103B1000010E1A6FD0EC2EF00101160E196F010E76
:103B20001A6FD0EC2EF00101150E196F010E1A6FED
:103B3000D0EC2EF001D0A3D074D0010E0101116F92
:103B400070D00101140E196F010E1A6FD0EC2EF017
:103B500001011451040AD8A401D001D036D0170EA7
:103B6000196F000E1A6FD0EC2EF00101160E196FAE
:103B7000000E1A6FD0EC2EF00101150E196F000E19
:103B80001A6FD0EC2EF00101140E196F000E1A6F8F
:103B9000D0EC2EF000EE17F0000EED5C08E1000E08
:103BA000ED5C05E1070EED5C02E1090EEF5CD8A0CB
:103BB00001D001D009D00001F80E1427F80E15230A
:103BC000FF0E1623FF0E172301D059D02AD0010172
:103BD000140E196F010E1A6FD0EC2EF007D00101F0
:103BE000130E196F010E1A6FD0EC2EF0010114079D
:103BF0001429D8A401D001D0F2D713D00101145157
:103C0000010A01E105D7020A01E12ED7300A99E045
:103C1000060A01E1E7D6030A01E163D7C90A8DE08C
:103C2000D6D701011151D8B401D001D0D3D60101AA
:103C30001251020AD8A401D001D009D015C118F040
:103C400016C119F017C11AF018C11BF013D000EEFD
:103C500018F00101EE50151908E1EE50161905E1B2
:103C6000EE50171902E1EE501819D8B401D001D066
:103C700001D0126B2CEC2FF00101125102D0000E7A
:103C800000D01200FFFF42D6FFFFD2D00101116F1A
:103C9000010EADEC2DF0010EADEC2DF0060EADECED
:103CA0002DF0000EADEC2DF0120EADEC2DF0230E2C
:103CB000ADEC2DF0340EADEC2DF0560EADEC2DF03C
:103CC000000EADEC2DF0000EADEC2DF0800EADEC45
:103CD0002DF0000EADEC2DF0000EADEC2DF0000E31
:103CE000ADEC2DF0000EADEC2DF0000EADEC2DF096
:103CF0000101126B00D0000EADEC2DF0010E0101A0
:103D000012270B0E126501D001D0F5D708C2E8FFCB
:103D1000ADEC2DF009C2E8FFADEC2DF00AC2E8FFD2
:103D2000ADEC2DF00BC2E8FFADEC2DF00CC2E8FFBE
:103D3000ADEC2DF00DC2E8FFADEC2DF00101126BE2
:103D400000D0000EADEC2DF0010E01011227C90EBE
:103D5000126501D001D0F5D7630EADEC2DF0820EC7
:103D6000ADEC2DF0530EADEC2DF0630EADEC2DF05F
:103D7000350EADEC2DF0010EADEC2DF00101115121
:103D8000ADEC2DF001011105D8B40AD000D000012E
:103D90002051211122112311D8B402D000D002D019
:103DA00000D016D0360EADEC2DF0040EADEC2DF09B
:103DB0001BC0E8FFADEC2DF01AC0E8FFADEC2DF014
:103DC00019C0E8FFADEC2DF018C0E8FFADEC2DF008
:103DD000370EADEC2DF0020EADEC2DF0010EADEC7A
:103DE0002DF0030EADEC2DF001011151030AD8A402
:103DF00001D001D016D0320EADEC2DF0040EADEC9A
:103E00002DF020C0E8FFADEC2DF021C0E8FFADECB7
:103E10002DF022C0E8FFADEC2DF023C0E8FFADECA3
:103E20002DF0FF0EADEC2DF035EC2EF01200FFFF63
:103E30002DD7FFFF16D00501716BFF0EE8CF57F2AB
:103E4000FF0EE8CF58F2FF0EE8CF59F2FF0EE8CF91
:103E50005AF2FF0EE8CF5BF2FF0EE8CF5CF21200E1
:103E6000FFFFE9D7FFFF53D049D00101070E116FC3
:103E7000010E126F060E136F010E146F71EC33F00A
:103E8000006E00C002F0036A03500210D8A401D0F3
:103E900001D001D038D001010651D8A401D001D001
:103EA00015D007C157F208C158F209C159F20AC129
:103EB0005AF20BC15BF20CC15CF20DC15DF20EC196
:103EC0005EF20FC15FF210C160F21DD0010EE8CFAB
:103ED00071F544EC26F00009D8B401D001D00BD024
:103EE0000101070E116F010E126F136B03EC34F01A
:103EF0000501716B02D0000E08D005D071C5E8FF36
:103F0000000AB3E0E6D7010E00D01200FFFFACD7E5
:103F10000001FFFF17D000C1E9FF01C1EAFFEECFAA
:103F200006F1EECF07F1EECF08F1EECF09F1010176
:103F3000000E116F010E126F010E136F03EC34F0BF
:103F40001200FFFFE8D70001FFFF43D000C1E9FFE7
:103F500001C1EAFF02015D51EE1808E15E51EE1861
:103F600005E15F51EE1802E16051EE18D8A401D0CE
:103F70001CD012C2E8FF5D6307D000D013C2E8FF77
:103F80005E6302D000D001D007D014C2E8FF020166
:103F90005F6302D000D001D007D015C2E8FF020154
:103FA000606302D000D001D001D002D000D00DD08B
:103FB000570EE96E020EEA6E02C1E1FF03C1E2FF95
:103FC000060EFAEC02F0010E02D0000E00D0120034
:103FD000FFFFBCD7FFFF02500002F3CF04F0F4CF85
:103FE00005F00102F350052603500002F3500526A8
:0A3FF0001200FFFF1200FFFFFDD7D3
:10400000FFFF28D00101006B00D0500E0101016FAD
:10401000026BF6EC05F0006E010100510A0D330E43
:10402000F324E96E020EF420EA6E00C0EFFF0051A7
:104030000A0D360EF324E96E020EF420EA6E000E2D
:10404000EF6E010E0027010E006501D001D0DDD713
:104050001200FFFFD7D7FFFF10D00101006B00D087
:10406000010100510BD8010E01010027010E00656E
:1040700001D001D0F5D71200FFFFEFD7FFFF89D2A3
:10408000D96ED9500A0D330EF3240101096F020EC7
:10409000F4200A6F010E026F74D20101026B09C194
:1040A000E9FF0AC1EAFFEF5043EC07F00009D8A48A
:1040B00001D001D00AD0010100EE03F00951E92638
:1040C0000A51EA22000EEF6E62D245D209C1E9FF21
:1040D0000AC1EAFFEF5030EC0AF00009D8B401D071
:1040E00001D0D4D0010E0101026F056B066B00D028
:1040F0000101000E065D500ED8B4055DD8A001D0B8
:104100001CD00551006E0651016E054B062B150E95
:104110000024666F010E0120676F09C1E9FF0AC123
:10412000EAFFEF50C8EC09F0006E00C002F0036A2D
:1041300003500210D8A402D000D002D000D0D8D7AB
:10414000010101EE15F00551E9260651EA22000EA3
:10415000EF6E09C1E9FF0AC1EAFFEF5047EC09F031
:10416000010100EE03F00951E9260A51EA22020E8C
:10417000EF6E050E036F150E666F010E676F0B0E67
:10418000686F010E696F030E6A6F010E6B6F090E87
:1041900009256C6F000E0A216D6F2BDB0101016F89
:1041A0000151D8A401D001D071D0010E036501D016
:1041B00001D011D00B0E666F010E676F0351686F4F
:1041C000EDEC16F0010100EE09F00951E9260A5163
:1041D000EA22030EEF6E0BC166F10CC167F123EC0E
:1041E00035F0010100EE01F00951E9260A51EA22F9
:1041F00000C0EEFF01C0EDFF09C1E1FF0AC1E2FF0F
:1042000000EE01F0E150E926E250EA22EE52ED50D4
:10421000FF0AFF0ED8B4EF18D8A401D001D011D0F6
:1042200000EE08F0E150E926E250EA22000EEF6EBF
:1042300000EE03F0E150E926E250EA22020EEF6EB2
:1042400025D000EE01F0E150E926E250EA22EE50DE
:10425000ED10D8A401D001D011D000EE08F0E1504B
:10426000E926E250EA22030EEF6E00EE03F0E15081
:10427000E926E250EA22020EEF6E08D000EE03F0CB
:10428000E150E926E250EA220B0EEF6E7AD109C125
:10429000E9FF0AC1EAFFEF509DEC08F00009D8B42D
:1042A00001D001D049D0010100EE08F00951E92602
:1042B0000A51EA22EF50020DE80EF324E96E000ED7
:1042C000F420EA6EEECF07F1EDCF08F10AD0D95015
:1042D00001016A6F09C1E9FF0AC1EAFFEF50C1ECB1
:1042E00008F0010107C1F6FF08C1F7FF010E07271B
:1042F000000E0823050EF76404D00800FFFFF550F8
:1043000005D0F6CFE9FFF7CFEAFFEF50D96ED950CD
:10431000D8A401D001D0DBD709C1E9FF0AC1EAFF67
:10432000EF50D2EC07F0010100EE03F00951E9264D
:104330000A51EA22090EEF6E24D109C1E9FF0AC130
:10434000EAFFEF509DEC08F00009D8B401D001D08D
:10435000AAD0010E0101026F046B00D004C100F06D
:10436000016A00507E0FF66E0150F76E070EF722BD
:104370000800FFFFF55001016A6F09C1E9FF0AC19A
:10438000EAFFEF50C1EC08F0010E010104271E0EF8
:10439000046501D001D0E2D7010100EE09F0095116
:1043A000E9260A51EA22EF50140DF20EF324076FAA
:1043B000060EF420086F0AD0D95001016A6F09C1B6
:1043C000E9FF0AC1EAFFEF50C1EC08F0010107C1A3
:1043D000F6FF08C1F7FF010E0727000E0823050EA0
:1043E000F76404D00800FFFFF55005D0F6CFE9FFD1
:1043F000F7CFEAFFEF50D96ED950D8A401D001D041
:10440000DBD70101046B00D004C100F0016A005049
:104410009E0FF66E0150F76E070EF7220800FFFFA1
:10442000F55001016A6F09C1E9FF0AC1EAFFEF50C7
:10443000C1EC08F0010E01010427030E046501D050
:1044400001D0E2D709C1E1FF0AC1E2FF00EE09F0A5
:10445000E150E926E250EA22EF50030AD8A401D045
:1044600001D009D000EE07F0E150E926E250EA223F
:10447000010EEF6E08D000EE07F0E150E926E250A1
:10448000EA22000EEF6E00EE04F0E150E926E25061
:10449000EA22030EEF6E00EE03F0E150E926E2504F
:1044A000EA22010EEF6E6DD009C1E9FF0AC1EAFFF1
:1044B000EF5030EC0AF00009D8B401D001D007D099
:1044C00009C1E9FF0AC1EAFFEF5047EC09F009C151
:1044D00066F10AC167F15FD8006E00C002F0036A9E
:1044E00003500210D8B401D001D00BD0BFEC35F08E
:1044F000010100EE03F00951E9260A51EA22090EF2
:10450000EF6E3FD009C1E9FF0AC1EAFFEF5043EC6B
:1045100007F00009D8B401D001D01CD009C1E9FFCF
:104520000AC1EAFFEF509DEC08F00009D8B401D0B1
:1045300001D010D009C1E9FF0AC1EAFFEF5057ECE2
:1045400007F0010100EE03F00951E9260A51EA22C1
:104550000A0EEF6E16D0010100EE03F00951E926B4
:104560000A51EA22EF50000A01E1B0D5010A9CE0AD
:10457000030A01E18CD60B0AC5E0020A01E1DDD68F
:1045800000D001010251D8A401D001D086D512007B
:10459000FFFF76D56601FFFF2AD1010100EE01F091
:1045A0006651E9266751EA22EECF6AF1EDCF6BF151
:1045B000D2EC35F0FFD00101686B00EE04F06651DB
:1045C000E9266751EA22EF50080AD8B401D001D099
:1045D00019D0ECEC35F00101696F02016451FF0A5A
:1045E000FF0ED8B46319D8A401D001D00BD01AECB7
:1045F00036F066C1E9FF67C1EAFFEF50D2EC07F081
:10460000010EF3D066C1E1FF67C1E2FF00EE07F0E3
:10461000E150E926E250EA22EF50D8B401D001D0AF
:10462000BFD09CD001016951250AD8A401D001D086
:1046300009D000EE04F0E150E926E250EA22050E2E
:10464000EF6E03D0010E0101686F9AD0010169512C
:10465000250AD8A401D001D00BD0010E686F00EE5E
:1046600004F0E150E926E250EA22030EEF6E12D088
:1046700000EE08F0E150E926E250EA220101693932
:10468000F00BEF6E00EE04F0E150E926E250EA2272
:10469000060EEF6E75D069C100F0D00E002600EE58
:1046A00008F0E150E926E250EA220050EF1200EE55
:1046B00004F0E150E926E250EA22080EEF6E00EE27
:1046C00005F0E150E926E250EA22000EEE6E000EFF
:1046D000ED6E56D0010100EE05F06651E9266751F6
:1046E000EA22EECF6AF1EDCF6BF1690E6C6F010E2D
:1046F0006D6F00EE08F06651E9266751EA22EF502F
:1047000046EC17F0010100EE05F06651E92667510D
:10471000EA2200C0EEFF01C0EDFF010E686F66C126
:10472000E1FF67C1E2FF00EE05F0E150E926E2504B
:10473000EA22EE52ED50FF0AFF0ED8B4EF18D8A4CB
:1047400001D001D008D000EE04F0E150E926E2509B
:10475000EA22030EEF6E14D000D0FFD700EE04F073
:10476000E150E926E250EA22EF50030A01E15AD76C
:10477000060A01E16BD7030A8EE00E0AABE0ECD724
:1047800001016851D8B401D001D009D069516A6FD4
:1047900066C1E9FF67C1EAFFEF50C1EC08F00AD03B
:1047A000010169516A6F66C1E9FF67C1EAFFEF5015
:1047B000C1EC08F066C1E9FF67C1EAFFEF509DEC6C
:1047C00008F00009D8A401D001D0F5D61AEC36F0D3
:1047D000010100EE01F06651E9266751EA2200C0AE
:1047E000EEFF01C0EDFF000E00D01200FFFFD5D696
:1047F0006601FFFF88D101016F6B746B756B706B85
:1048000066C176F167C177F1A30E786F070E796FF5
:10481000030E7A6F7B6B49EC3DF001500010D8A479
:1048200001D001D00BD066C1E1FF67C1E2FF040EE9
:10483000E126000EE22201016E6B02D0020E61D170
:1048400001D0E652E750200AD8B401D001D0F9D700
:10485000E750D96EBDD06AC1E9FF6BC1EAFFEF50E6
:104860000101705DD8A001D001D001D0CBD09ED085
:104870000101D8907035006E016A0136D9500024CC
:10488000E96EDA500120EA6EE1CFEEFFE2CFEDFFF4
:10489000E750D96ED9502F0AD8A401D005D0D950ED
:1048A0005C0AD8A402D000D002D000D003D0010E00
:1048B00001016F6F8AD00101D8907035006E016AD6
:1048C0000136D9500024E96EDA500120EA6EE1CFBA
:1048D000EEFFE2CFEDFF010E7027020E6F6FE75083
:1048E000E96EE9503F0AD8A401D005D0E950260A64
:1048F000D8A402D000D002D000D006D0000EE76EBF
:10490000010E01016F6F51D0E9502B0AD8A401D0DC
:1049100001D003D0200EE76E48D0E9502E0AD8A46B
:1049200007D000D001017005D8A402D000D002D079
:1049300000D006D0E652E1CF74F1E2CF75F135D068
:10494000E9503D0AD8A401D001D006D0000EE76E90
:10495000010E01016F6F29D0E9502F0AD8A401D0B0
:1049600005D0E9505C0AD8A402D000D002D000D013
:104970001CD0010EE1CF00F0E2CF01F00026000EC6
:1049800001220101D8907035026E036A0336D950B6
:104990000226DA500322FE0E0224E96EFF0E0320E7
:1049A000EA6E00C0EEFF01C0EDFF0FD068C1D9FF75
:1049B00069C1DAFF01016F51000A01E159D7010A0B
:1049C00001E179D7030A8BE000D0E652E750D96EB7
:1049D000D950200AD8A401D004D0D950D8A402D0EC
:1049E00000D006D000D0D9500D0AD8A402D000D0F3
:1049F00006D000D0D9500A0AD8A402D000D002D0E4
:104A000000D029D7000EE76E6CC1E9FF6DC1EAFF47
:104A1000070EEF6E010175517411D8B401D001D0A9
:104A200038D074C17AF175C17BF1AAEC3AF000C0BC
:104A300074F101C075F10101D60E726F060E736F2D
:104A4000716B00D074C176F175C177F172C178F1E4
:104A500073C179F1030E01017A6F7B6B49EC3DF074
:104A600001500010D8A401D001D007D06CC1E9FFDB
:104A70006DC1EAFF71C1EFFF0CD0040E0101722776
:104A8000000E7323010E7127060E716501D001D04F
:104A9000D9D701017051D8A401D001D029D068C163
:104AA000E9FF69C1EAFFEECF76F1EDCF77F1A70E0E
:104AB000786F070E796F090E7A6FCFEC3AF068C104
:104AC000E9FF69C1EAFFEECF00F0EDCF01F0090E7A
:104AD0000024E96E000E0120EA6E000EEF6E6CC13C
:104AE000E9FF6DC1EAFF010EEF6E010E01017027B3
:104AF0006AC1E9FF6BC1EAFF70C1EFFF01016E51AE
:104B000000D01200FFFF77D6FFFFBDD0D96A00D0DA
:104B1000D950020D6B0EF324E96E020EF420EA6EFA
:104B2000D9CF00F0D8900036D8900034400FEF6E07
:104B3000D950020D6C0EF324E96E020EF420EA6ED9
:104B4000010EEF6E010ED926000ED96401D001D0FE
:104B5000DFD70501A96B2EDB020EACEC3EF01F0E79
:104B60004FDB0101D16F1F0E3CDB020EACEC3EF0BF
:104B7000070E46DB006E00AE01D001D082D0210EC0
:104B80000101D16F000E2DDB020EACEC3EF0480EA1
:104B90000101D16F0E0E25DB0101D16B0A0E21DB65
:104BA0000101D16B0B0E1DDB040E0101D16F0C0E48
:104BB00018DB020E0101D16F0D0E13DBA9C5E8FF52
:104BC000020D6B0EF324E96E020EF420EA6EEF5034
:104BD0000101D16F040E05DB440E0101D16F010EFE
:104BE00000DB5F0E0101D16F020EFBDA5E0E0101E8
:104BF000D16F030EF6DA0101D169070EF2DA010175
:104C0000D16B0F0EEEDA610E0101D16F000EE9DA01
:104C100008C2D1F1010EE5DA09C2D1F1020EE1DAE2
:104C20000AC2D1F1030EDDDA0BC2D1F1040ED9DADA
:104C30000CC2D1F1050ED5DA0DC2D1F1060ED1DAD2
:104C40000101006B00D00101D1690051080FC9DAE0
:104C5000010E01010027070E006501D001D0F3D736
:104C6000440E0101D16F070EBCDA440EE8CFAAF55D
:104C7000220E0101D16F000EB4DA0101D16B0D0ECD
:104C8000B0DA1200FFFF42D7FFFF09D0000EB8DAFA
:104C9000006E000E00A4010E00D01200FFFFF6D738
:104CA000FFFF17D00101CB6F010E0101D16F0A0E7A
:104CB00098DA0101D16B0B0E94DA120E0101D16F5B
:104CC000000E8FDA0101CB51D16F100E8ADA12007B
:104CD000FFFFE8D7CB01FFFF59D0010ECDC100F097
:104CE000CEC101F00016000E01160101CD510024C5
:104CF000CF6FCE510120D06F400ED16F070E71DA09
:104D00000101CF51D16F0A0E6CDA0101D051D16F80
:104D10000B0E67DA120E0101D16F000E62DA0DD0B0
:104D2000CBC1E9FFCCC1EAFFEF500101D16F010E09
:104D3000CB27000ECC23100E54DA0101CD51006EAA
:104D4000CE51016E010ECD5F000ECE5B0150001002
:104D5000D8A401D001D0E4D7FF0E0101CD6FCE6BF6
:104D600004D00101CD07D8A0CE070101CE51CD114D
:104D7000D8A401D006D0070E43DA006E00AC02D0F2
:104D800000D002D000D0EDD71200FFFFA6D7FFFF62
:104D900013D0010E0101D16F0A0E23DA0101D16B8C
:104DA0000B0E1FDA0A0E0101D16F000E1ADA100E77
:104DB00027DA00D01200FFFFECD74001FFFF3BD005
:104DC00042C144F143C145F1400E0101D16F070ECC
:104DD00008DA01014451D16F0A0E03DA010145518D
:104DE000D16F0B0EFED90A0E0101D16F000EF9D959
:104DF0000CD0100E05DA40C1E9FF41C1EAFFEF6EA9
:104E0000010E01014027000E412301014251006EB5
:104E10004351016E010E425F000E435B01500010D2
:104E2000D8A401D001D0E5D744C100F045C101F0BC
:104E300000D01200FFFFC4D7FFFF0DD0D96ED950AC
:104E4000020D6C0EF324E96E020EF420EA6E000EE1
:104E5000EF6E1200FFFFF2D7FFFF0FD0D96ED950CF
:104E6000020D6C0EF324E96E020EF420EA6E010EC0
:104E7000EF6ED9CFA9F51200FFFFF0D7FFFF18D0D2
:104E80000501AA0501016B6F440E6B6101D001D0D1
:104E900002D05E0E6B6F200E0101D16F000EA1D902
:104EA00001016B51D16F030E9CD900D01200FFFF9E
:104EB000E7D7FFFF2FD0600E0101D16F000E91D90F
:104EC000070E9ED90101AA6F200ED16F000E89D95D
:104ED000A8C5E8FF0101AA6101D001D008D0A8C58A
:104EE000E8FF5F08006EAA510024D96E05D0A8C55E
:104EF000E8FF0101AA5DD96ED9501B08D96ED950BF
:104F00000101AC6FAB6BABC100F0ACC101F000D0E4
:104F10001200FFFFD0D70601FFFFB3D008C1E9FFA1
:104F200009C1EAFFFF0EEF6E070E6AD9006E00A8F6
:104F300001D001D024D0210E0101D16F000E51D932
:104F4000FF0E86D90101D16B0A0E4BD90101D16B3D
:104F50000B0E47D9020E0101D16F0D0E42D9200E62
:104F60000101D16F000E3DD989DF0101D169070E22
:104F700038D90101D16B0D0E34D9000E80D0600EEE
:104F80000101D16F000E2DD9070E3AD901010A6F28
:104F9000200ED16F000E25D901010A510501AA1971
:104FA000D8B401D001D069D0AAC50CF101010B6BB6
:104FB0000BC1CBF10CC1CCF133D901010D0E406F07
:104FC000010E416F120E426F436BF8DE01010DA11D
:104FD0000DD000D001EE0FF0EE52000EED5C400E51
:104FE000D8B4EF5CD8A002D000D001D00CD001EE34
:104FF0000FF0EE52050EED5CEF0ED8B4EF5CD8B0BA
:1050000002D000D002D000D032D01DC1C5F11EC1E7
:10501000C6F1D3EC39F000C01DF101C01EF106C18C
:1050200046F107C147F10101170E486F010E496FA4
:10503000060E4A6F4B6BE5EC3DF001011E51080A6C
:10504000D8A40DD000D01D51D8A401D005D01D5139
:10505000060AD8A402D000D001D001D002D000D0DE
:1050600006D008C1E9FF09C1EAFF1DC1EFFFAAC5CB
:10507000A8F50EC1AAF5010E02D0000E00D0120054
:10508000FFFF4CD7C301FFFF63D00A0E0101D16FB0
:10509000070EA7D8A9C5E8FF020D6B0EF324E96E31
:1050A000020EF420EA6EEF500101CA6FC96BC9C14C
:1050B000CBF1CAC1CCF1B4D8C3C1CBF1C4C1CCF1DE
:1050C000060E0101CD6FCE6B06DE08C2E8FFE8DDFB
:1050D00009C2E8FFE5DD0AC2E8FFE2DD0BC2E8FF36
:1050E000DFDD0CC2E8FFDCDD0DC2E8FFD9DD010128
:1050F000C551D8A401D001D002D0C86B03D0060E90
:105100000101C86F080ECCDD0101C851C9DD0E0ECA
:105110000101C627000EC723000EC75D3C0ED8B4A0
:10512000C65DD8B001D001D003D0400EC66FC76BAA
:10513000C6C1C9F1C7C1CAF10101C951D16F050E7C
:1051400050D80101CA51D16F060E4BD81200FFFF93
:105150009CD7FFFF2ED0A9C5E8FF020D6B0EF324EC
:10516000E96E020EF420EA6EEF500101D16F040ED9
:1051700038D8240E0101D16F000E33D8D96A00D07F
:10518000D950020D6C0EF324E96E020EF420EA6E83
:10519000EF50D8B401D001D003D0D9CFA9F507D0B2
:1051A000010ED926000ED96401D001D0E9D7120032
:1051B000FFFFD1D7FFFF13D09568816AE00E936E91
:1051C000F19E848284808484966A00D0010ED96E18
:1051D00001D000D0D92EFDD784941200FFFFECD768
:1051E000D101FFFF0CD0816EE00E936E0101D15111
:1051F000836E956A8492848295681200FFFFF3D7CC
:10520000FFFF0CD09568816EE00E936E8490835002
:10521000D96E8480D95000D01200FFFFF3D7CB01A4
:10522000FFFF15D0CBC1CDF1CCC1CEF1400E0101B5
:10523000D16F070ED6DF0101CD51D16F080ED1DF3E
:105240000101CE51D16F090ECCDF1200FFFFEAD76A
:10525000FFFF15D00101206F1F6B00D001011F510E
:10526000006E2051016E010E1F5F000E205B015089
:105270000010D8A401D001D0F1D71200FFFFEAD767
:105280006A01FFFF10D0A8C56DF1120E01016C6F0D
:105290006A516C276B516D236CC1CBF16DC1CCF1A0
:1052A000BFDF1200FFFFEFD7AA01FFFF1BD0E8CF3F
:1052B000A9F5A9C5E8FF020D6B0EF324E96E020EF5
:1052C000F420EA6EEF500101AD6F0E0EAC6FAA51E3
:1052D000AC27AB51AD23ACC1CBF1ADC1CCF1A0DF5C
:1052E0001200FFFFE4D7FFFF0FD0090E89DF010195
:1052F000016F080E85DF0101006F00C100F001C1E0
:1053000001F000D01200FFFFF0D7FFFF15D0150EFF
:105310000101016F026BF6EC05F0E8CF78F50501AD
:105320007B6B0501796B0501766B0201140E1D6F15
:10533000000E1E6F1200FFFFEAD7FFFF51D178C5A4
:10534000E8FF43EC07F00009D8A401D001D00DD04C
:105350000501796B070EE8CF74F505017B6B05013C
:10536000766B05017C6B010E39D178C5E8FF30EC16
:105370000AF00009D8B401D001D052D05DEC3EF063
:1053800000C021F201C022F202C023F203C024F2C5
:1053900015D079C5E8FF05EE87F0E926000EEA2270
:1053A00000C1EFFF0501010E792779C5E8FF1F0A4B
:1053B000D8A401D001D002D00501796B0101000E03
:1053C000666F010E676F78C5E8FFC8EC09F0006EE4
:1053D00000C002F0036A03500210D8A401D001D02B
:1053E000D8D778C5E8FF47EC09F0010100510A0A57
:1053F000D8A401D001D013D079C5E8FF05EE87F01D
:10540000E926000EEA22000EEF6E0501796B9BDAA9
:1054100025C207F126C208F165DAE8CF74F542D05B
:1054200005017B53D8B401D001D03CD05DEC3EF0F7
:1054300000C001F101C002F102C003F103C004F198
:10544000010EE96E010EEA6E21C2E8FFEE5E22C295
:10545000E8FFEE5A23C2E8FFEE5A24C2E8FFED5AF5
:10546000ED52ED520101000E045D08E1000E035DF6
:1054700005E1460E025D02E1500E015DD8A001D0AB
:1054800001D010D05DEC3EF000C021F201C022F24C
:1054900002C023F203C024F2020EE8CF74F5010E1D
:1054A000E8CF7BF58ED00501776B5DEC3EF000C058
:1054B00021F201C022F202C023F203C024F200D084
:1054C00078C5E8FF9DEC08F00009D8B401D001D000
:1054D000F7D778C5E8FF9DEC08F00009D8B401D0F3
:1054E00001D03AD077C5E8FF020DD20EF324E96E61
:1054F000000EF420EA6EEECF05F1EDCF06F107D0F5
:10550000010100516A6F78C5E8FFC1EC08F00101A4
:1055100005C1F6FF06C1F7FF010E0527000E0623A1
:10552000050EF76404D00800FFFFF55005D0F6CF54
:10553000E9FFF7CFEAFFEF50006F0051D8A401D088
:1055400001D0DED778C5E8FFD2EC07F00B0EE8CF2C
:1055500077F5010EE8CF7BF574C5E8FF070AD8B4EC
:1055600001D001D02DD074C5E8FF3BD80009D8B4D4
:1055700001D001D01AD077C5E8FF0B0AD8B401D00A
:1055800001D004D0040EE8CF7BF509D074C5E8FF44
:10559000020AD8A401D001D002D005017B6B070E0E
:1055A000E8CF74F505017C6B0BD077C5E8FF0B0ADB
:1055B000D8B401D001D004D0040EE8CF7BF57FD75A
:1055C0000BD07BC5E8FF000A01E16DD7010AC4E0FA
:1055D000050A01E174D700D0010E00D01200FFFFD0
:1055E000AED6FFFF82D0D96E6ED00501768105015F
:1055F0007693010EE8CF77F501017D0E076F050E5A
:10560000086F01EE09F027C2EEFF28C2EDFF0A0E77
:105610000B6F0C6BA0EC3DF064D076C500F000B0D1
:1056200001D001D004D0060EE8CF77F520D00101DB
:105630007D0E076F050E086F01EE09F027C2EEFF21
:1056400028C2EDFFAFEC17F0006E00C002F0036A55
:1056500003500210D8B401D001D006D005017683E2
:10566000020EE8CF77F503D0060EE8CF77F539D0F4
:105670003DD839D02FC226F130C227F128EC3CF0BA
:1056800000C01EF231C226F132C227F128EC3CF0F4
:1056900000C01DF20A0EE8CF77F523D07BD823D0C7
:1056A0000A0EE8CF77F575C5E8FFFE0AD8B401D039
:1056B00001D004D075C5E8FF57EC07F012D0050EF5
:1056C000E8CF77F50ED0D950000A8FE0010AA5E0A7
:1056D000030ACEE0010AE2E0070ACCE0010AE0E0BA
:1056E000EED7010E00D01200FFFF7DD7FFFF51D093
:1056F00043D07CC5E8FF020AD8A401D001D002D073
:10570000BFEC35F075C5E8FFFE0AD8B401D001D072
:105710000AD0BFEC35F075C5E8FF57EC07F0010E75
:10572000E8CF7CF501D00AD030D075C5E8FF43EC56
:1057300007F00009D8A401D001D006D0030EE8CFAD
:1057400077F5030EE8CF7CF520D078C5E8FF9DEC17
:1057500008F00009D8B401D001D00DD078C5E8FF19
:1057600043EC07F00009D8B401D001D004D078C5CB
:10577000E8FF57EC07F009D07CC5E8FF000AB9E064
:10578000010AD3E0020AE1E000D0000E00D01200CE
:10579000FFFFAED7FFFFA4D095D076C500F000B2D2
:1057A00001D001D005D0060EE8CF77F5010E96D0D6
:1057B000070EE8CF77F578C5E8FF260D2F0EF32406
:1057C0000101086F000EF420096F01EE0AF01DC2FE
:1057D000EEFF1EC2EDFF5EEC06F0E8CF75F5010EA0
:1057E000E8CF7CF579D075C5E8FF43EC07F00009F8
:1057F000D8B401D001D00FD00501AD53D8A401D049
:1058000001D009D026EC36F000C01FF201C020F212
:10581000020EE8CF7CF560D075C5E8FF30EC0AF0E9
:105820000009D8B401D001D033D05DEC3EF000C007
:1058300021F201C022F202C023F203C024F21FC2EF
:10584000ADF120C2AEF132EC36F004D001010751C7
:1058500051EC36F00101070E666F010E676F75C5DA
:10586000E8FFC8EC09F0006E00C002F0036A0350C4
:105870000210D8A401D001D0E9D77BEC36F000C0EB
:105880001FF201C020F275C5E8FF47EC09F019D0FE
:1058900075C5E8FF43EC07F00009D8A401D001D09A
:1058A00010D07BEC36F0BFEC35F075C5E8FF57EC57
:1058B00007F0FE0EE8CF75F5090EE8CF77F5010E7B
:1058C0000DD00AD07CC5E8FF000A01E166D7010AC5
:1058D0008AE0030AA1E000D0000E00D01200FFFF12
:1058E0005BD70701FFFF2ED00101096B00D007C174
:1058F00076F108C177F101010951020DC60EF324BA
:10590000E96E000EF420EA6EEECF78F1EDCF79F17A
:10591000040E7A6F7B6B49EC3DF001500010D8A467
:1059200001D001D003D0010109510AD0010E0101BB
:105930000927050E096501D001D0D9D7060E00D080
:105940001200FFFFD1D7FFFF60D0E96A870EE16E3A
:10595000050EE26E01D0E652E750200AD8B401D01D
:1059600001D0F9D7E1CF25F2E2CF26F2010EE8CF40
:105970007AF542D03AD0D950200AD8A401D005D027
:10598000D9502C0AD8A402D000D002D000D005D023
:10599000000EE76E010EE96E0FD0D9500D0AD8A4A3
:1059A00001D005D0D9500A0AD8A402D000D002D024
:1059B00000D002D0000EE76E1ED0D950200AD8B415
:1059C00001D001D011D07AC5E8FF020D250EF324D5
:1059D000E96E020EF420EA6EE1CFEEFFE2CFEDFFBA
:1059E0000501010E7A27E96A06D0E950000AC3E0F2
:1059F000010AE3E000D0E652E750D96ED950D8A4AE
:105A000001D001D0B7D71200FFFF9FD7FFFF21D0F1
:105A1000D96A00D0D950160DDE0EF324E96E010EBE
:105A2000F420EA6EFF0EEE6E000EED6ED950160DEC
:105A3000E70EF324E96E010EF420EA6EFE0EEF1677
:105A4000010ED926010ED96401D001D0E3D712008E
:105A5000FFFFDED71101FFFF6DD0D20EE16E010E08
:105A6000E26E0101176B00D000EE0CF0E150E92668
:105A7000E250EA22EE50FF0AED10D8A401D001D086
:105A800049D000EE0CF0E150E926E250EA2211C1C3
:105A9000EEFF12C1EDFFE1CF18F1E2CF19F10101E4
:105AA00014511311D8B401D001D00DD018C146F152
:105AB00019C147F113C148F114C149F10A0E4A6FE7
:105AC0004B6BE5EC3DF018C1E1FF19C1E2FF00EEC0
:105AD0000AF0E150E926E250EA2215C1EEFF16C1B4
:105AE000EDFF00EE0EF0E150E926E250EA22000E52
:105AF000EE6E000EED6E00EE10F0E150E926E25081
:105B0000EA22000EEE6E000EED6E17C1D0F5010117
:105B100017510ED0160EE126000EE222010E0101F1
:105B20001727010E176501D001D09ED7FF0E00D0B8
:105B30001200FFFF92D7FFFF0FD0D96ED950160D7C
:105B4000DE0EF324E96E010EF420EA6EFF0EEE6E17
:105B5000000EED6E1200FFFFF0D7FFFF85D00101B0
:105B6000136FD0C5E8FF160DD20EF324D96E010EC7
:105B7000F420DA6ED9CF14F1DACF15F100EE0EF081
:105B8000D950E926DA50EA22EE50ED10D8A401D01F
:105B900001D020D0010100EE12F01451E926155178
:105BA000EA22A9C5EFFF1C0EAA6FAB6B00EE12F044
:105BB0001451E9261551EA22EF5055EC29F0010164
:105BC00000EE13F01451E9261551EA22000EEE6E94
:105BD000000EED6E0101135150EC26F014C1E1FFEF
:105BE00015C1E2FF00EE0EF0E150E926E250EA2294
:105BF000EECF00F0EDCF01F000EE13F0E150E9261A
:105C0000E250EA22EFCF02F0010EEE26EFCF03F0D2
:105C1000000EED220150035C02E10050025CD8A0AE
:105C200001D001D009D000EE0EF0E150E926E2509B
:105C3000EA22EE2A000EED2200EE0EF0E150E926F7
:105C4000E250EA22EECFF3FFEDCFF4FF030EF45C57
:105C5000D60ED8B4F35CD8A001D001D001D005D8BD
:105C6000010E00D01200FFFF7AD7FFFF85D0D0C50C
:105C7000E8FF160DD20EF3240101166F010EF42079
:105C8000176F00EE0CF01651E9261751EA22EECFFD
:105C9000C5F1EDCFC6F1D3EC39F000C018F101C069
:105CA00019F1010100EE0AF01651E9261751EA2216
:105CB000EECFC5F1EDCFC6F1D3EC39F000C01AF14B
:105CC00001C01BF1010100EE0EF01651E92617513B
:105CD000EA22EECF00F0EDCF01F0080E00241C6F99
:105CE000000E01201D6F1E6B1F6B140EAA6FAB6B95
:105CF00000EE12F01651E9261751EA22EF5055EC4A
:105D000029F016C1AAF117C1ABF1110E0101AC6F58
:105D10001CC1ADF11DC1AEF195EC37F01CC1C5F150
:105D20001DC1C6F1D3EC39F000C01CF101C01DF15A
:105D30000101180ECB6F010ECC6F080ECD6FCE6B2C
:105D40006BEC26F0A9EC28F016C1E1FF17C1E2FFC9
:105D500000EE12F0E150E926E250EA22FF0EEF6E6B
:105D600000EE0EF0E150E926E250EA22000EEE6E5F
:105D7000000EED6E1200FFFF7AD7FFFF0FD0E8CFC5
:105D8000D0F5D0C5E8FF160DE20EF324E96E010E42
:105D9000F420EA6EEF5000D01200FFFFF0D7190197
:105DA000FFFF59D0D0C5E8FF160DE20EF324E96ECF
:105DB000010EF420EA6EEE50ED10D8A401D001D00F
:105DC00002D0000E46D0D0C5E8FF160DE70EF32432
:105DD000E96E010EF420EA6EEF50006E00A001D0D3
:105DE00001D011D0D0C5E8FF160DE70EF324E96EFF
:105DF000010EF420EA6EFE0EEF161C0E01016A6F12
:105E00006B6B41EC29F0C7EC26F019C1E9FF1AC110
:105E1000EAFFEF6ED0C5E8FF160DE20EF324E96E3F
:105E2000010EF420EA6EEE06000EED5AD0C5E8FF32
:105E3000160DE20EF324E96E010EF420EA6EEE5028
:105E4000ED10D8A401D001D002D03EEC27F0010E15
:105E500000D01200FFFFA6D7FFFF20D0D0C5E8FF7B
:105E6000160DE20EF324E96E010EF420EA6EEE50F8
:105E7000ED10D8B401D001D002D03EEC27F0D0C54F
:105E8000E8FF160DE20EF324E96E010EF420EA6E2F
:105E9000000EEE6E000EED6E1200FFFFDFD7060162
:105EA000FFFF66D001010B0E406F010E416F080E1F
:105EB000426F436BDEEC26F00BC1C5F10CC1C6F19D
:105EC000D3EC39F000C00BF101C00CF10DC1C5F1EC
:105ED0000EC1C6F1D3EC39F000C00DF101C00EF1D6
:105EE0000FC1C5F110C1C6F1D3EC39F0F80E002492
:105EF00001010F6FFF0E0120106F11C1C5F112C11A
:105F0000C6F1D3EC39F000C011F101C012F101016A
:105F10000B0E136F010E146F06C115F107C116F1B8
:105F200029D801010A6F0A29D8A401D001D003D0D1
:105F30003EEC27F019D001010A51160DE20EF324B0
:105F4000E96E010EF420EA6E0FC1EEFF10C1EDFF05
:105F50000A51160DE70EF324E96E010EF420EA6EE5
:105F6000EF50FE0B0109EF6E010E00D01200FFFF93
:105F700099D71301FFFFB9D001011769D20ED96E6D
:105F8000010EDA6EF36A00D0010110EE02F0135137
:105F9000E1261451E22200EE0CF0D950E926DA5045
:105FA000EA22EE52E652E550ED18E7CFE8FFD8B40A
:105FB000EF18D8A401D001D05AD013C1E9FF14C101
:105FC000EAFF10EE0AF0D950E126DA50E222E6525A
:105FD000EE52ED50E518EFCFE8FFD8B4E718D8A49B
:105FE0000DD000D000EE10F0D950E926DA50EA22A8
:105FF000EE50ED10D8A402D000D002D000D034D0A2
:10600000010110EE06F01551E1261651E22200EED4
:1060100006F0D950E926DA50EA22EE50E61808E1F7
:10602000EE50E61805E1EE50E61802E1EE50E618F3
:10603000D8A401D014D000EE06F0D950E926DA50E9
:10604000EA22FF0EEE18FF0ED8B4EE18FF0ED8B4F9
:10605000EE18FF0ED8B4EE18D8A402D000D002D0AB
:1060600000D002D0F3503FD0F3500101176F160E4D
:10607000D926000EDA22010EF326010EF36401D0B8
:1060800001D082D701011729D8B401D001D028D07E
:106090001751160DD20EF324E96E010EF420EA6EAC
:1060A000E9CF46F1EACF47F1E9CF18F1EACF19F18C
:1060B00015C148F116C149F10A0E4A6F4B6BE5EC68
:1060C0003DF013C1E9FF14C1EAFF010110EE0AF02F
:1060D0001851E1261951E222EECFE6FFEDCFE5FFA0
:1060E0000101175100D01200FFFF46D72B01FFFF1F
:1060F0000101396B3A6B2BC137F12CC138F1010129
:106100002FC1F6FF30C1F7FF2F2B000E3023050EF5
:10611000F76404D00800FFFFF55005D0F6CFE9FF83
:10612000F7CFEAFFEF50346F34510101D8B4C7D232
:10613000250AD8B40BD0392B000E3A232E512D113D
:10614000D8A47BD13451F9EC1FF0D9D701013269C1
:10615000336B316B62D201012E512D11D8A4B3D211
:10616000B8D237C1E9FF38C1EAFF0101020E372773
:10617000000E3823EF5095D20101318D4ED201012E
:10618000312B06D0080E01013227FE0E0101322705
:1061900037C1E9FF38C1EAFF0101020E3727000EBF
:1061A0003823EECF35F1EDCF36F131A10DD036AF3A
:1061B00006D0356D361FD8B0362B330707D0010116
:1061C000319131AD03D0F9D7010131910B0E0101AD
:1061D000322732C102F0036A35C100F036C101F046
:1061E0001BEC3EF000500101346F32C102F0036A33
:1061F00035C100F036C101F01BEC3EF004C035F1B2
:1062000005C036F1010E3B6F3C6B01013C51365D20
:1062100002E13B51355DD8A010D032C102F0036AD3
:106220003BC100F03CC101F0EAEC1FF004C03BF1BF
:1062300005C03CF101013307E8D7010131A916D0AF
:106240001CD00101392B000E3A232E512D11D8B448
:106250000AD02DC1E9FF2EC1EAFF200EEF6E2D2BD3
:10626000000E2E2303D0200EF9EC1FF0010133079E
:106270003351800A7F0FD8B0E4D7010131A115D086
:10628000392B000E3A232E512D11D8B40AD02DC12E
:10629000E9FF2EC1EAFF2D0EEF6E2D2B000E2E23EF
:1062A00017D02D0EF9EC1FF013D0010131AD10D035
:1062B000392B000E3A232E512D11D8B406D02DC102
:1062C000E9FF2EC1EAFF2B0EE7D72B0EF9EC1FF0EA
:1062D000010131B916D051D00101392B000E3A23FA
:1062E0002E512D11D8B40AD02DC1E9FF2EC1EAFFDD
:1062F000300EEF6E2D2B000E2E2303D0300EF9EC56
:106300001FF0010133073351800A7F0FD8A035D029
:10631000E3D73BC102F03CC103F035C100F036C108
:1063200001F01BEC3EF004C000F005C001F032C1EA
:1063300002F0036A1BEC3EF000500101336F800A4B
:10634000760FD8A002D0070E33270101392B000E9B
:106350003A232E512D11D8B40BD03351300F2DC10B
:10636000E9FF2EC1EAFFEF6E2D2B000E2E2305D084
:1063700001013351300FF9EC1FF032C102F0036A12
:106380003B0EE96E010EEA6EEE50006EEF50016EAC
:106390001BEC3EF00550ED6E0450EF6EEE50ED102C
:1063A000D8A4B7D7090E0101346502D0070E3427EF
:1063B0000101392B000E3A232E512D11D8B408D0EB
:1063C0003451300F2DC1E9FF2EC1EAFFEF6E3BD0F3
:1063D00001013451300FF9EC1FF091D60101335116
:1063E000800A7E0FD8A017D0392B000E3A232E51E9
:1063F0002D11D8B40AD02DC1E9FF2EC1EAFF200E1D
:10640000EF6E2D2B000E2E2303D0200EF9EC1FF083
:1064100001013307E3D737C1E9FF38C1EAFF0101C2
:10642000020E3727000E3823EF50346F392B000E41
:106430003A232E512D11D8B40AD02DC1E9FF2EC117
:10644000EAFF34C1EFFF2D2B000E2E2358D6010199
:106450003451F9EC1FF053D637C1E9FF38C1EAFFD8
:106460000101020E3727000E3823EECF00F0EDCFEA
:1064700001F000C0FEF101C0FFF1D96AFEC100F0D9
:10648000FFC101F0D9500024026E000E0120036EFE
:1064900002C0F6FF03C0F7FF050EF76404D0080042
:1064A000FFFFF55005D0F6CFE9FFF7CFEAFFEF5039
:1064B0000009D8B402D0D92AE1D701013251D960FC
:1064C00002D0D950326F0101325133BF46D0FF0A9A
:1064D0003325D8A042D0392B000E3A232E512D114E
:1064E000D8B40AD02DC1E9FF2EC1EAFF200EEF6E0D
:1064F0002D2B000E2E2303D0200EF9EC1FF00101EE
:106500003307E1D7FEC1F6FFFFC1F7FF050EF764C1
:1065100004D00800FFFFF55005D0F6CFE9FFF7CF14
:10652000EAFFEF500101346F0101FE2B000EFF2343
:106530000101392B3A232E512D11D8B40AD02DC187
:10654000E9FF2EC1EAFF34C1EFFF2D2B000E2E23F1
:1065500004D001013451F9EC1FF001013207322956
:10656000D8B4CDD5CFD72FC1F6FF30C1F7FF050E78
:10657000F76404D00800FFFFF55005D0F6CFE9FF1F
:10658000F7CFEAFFEF502A0AD8A40FD037C1E9FFAE
:1065900038C1EAFF0101020E3727000E3823EF5001
:1065A000326F2F2B000E302338D02FC1F6FF30C1B1
:1065B000F7FF050EF76404D00800FFFFF55005D083
:1065C000F6CFE9FFF7CFEAFFEF50D00F0101326FAE
:1065D0002F2B000E30232FC1F6FF30C1F7FF050E21
:1065E000F76404D00800FFFFF55005D0F6CFE9FFAF
:1065F000F7CFEAFFEF50D96E2F0ED9640ED03A0EC6
:10660000D9600BD0010132510A0DD950F324D00FBB
:10661000C7D7010131B538D0318901012FC1F6FF4B
:1066200030C1F7FF2F2B000E3023050EF76404D086
:106630000800FFFFF55005D0F6CFE9FFF7CFEAFFDE
:10664000EF50346F000A01E186D52A0A01E189D5AD
:10665000010A01E191D5050A86E01E0ADAE0680A1E
:1066600001E190D53B0A01E1B9D6070A01E187D5DE
:106670000B0A01E18AD51C0A01E1EED6060A01E106
:1066800087D50D0A01E17ED52F0E010134650BD0AF
:106690003A0E346108D0318533510A0D3451F32458
:1066A000D00F336FBAD70101392B000E3A232E5188
:1066B0002D11D8A4C2D63451F9EC1FF020D52E519B
:1066C0002D11D8B406D02DC1E9FF2EC1EAFF000E6E
:1066D000EF6A39C100F03AC101F01200FFFF08D59E
:1066E0001101FFFF8ED00101150E406F010E416FA9
:1066F0001C0E426F436BDEEC26F03EEC27F00101EE
:10670000150E316F010E326F49D901EE15F0EE50C2
:10671000010AED10D8B401D006D001011951060AC2
:10672000D8B402D000D007D000D001011A51040A19
:10673000D8B402D000D002D000D002D0000E5FD07A
:1067400013C1E1FF14C1E2FF11C1D9FF12C1DAFF89
:1067500001EE1BF0EE50020AED10D8A401D001D0DA
:1067600003D0000EE76E10D001EE1BF0EE50010AD0
:10677000ED10D8A401D001D003D0010EE76E04D0F3
:10678000020EE76E000E3BD004C2E8FF01012D634C
:1067900007D000D005C2E8FF2E6302D000D001D0A0
:1067A00007D006C2E8FF01012F6302D000D001D05C
:1067B00007D007C2E8FF0101306302D000D002D049
:1067C00000D01BD01D0EE96E010EEA6ED9CFE1FF9D
:1067D000DACFE2FF060EFAEC02F000EE06F0D95036
:1067E000E926DA50EA2223C1EEFF24C1EEFF25C1DB
:1067F000EEFF26C1EEFF010E02D0000E00D0120007
:10680000FFFF71D71101FFFFC7D0010E0101146F07
:10681000156B000E166F080E176F060E186F040E1C
:10682000196F11C1D9FF12C1DAFF1305D8A401D025
:1068300001D00AD0010E1A6F1B6B266927692869DF
:1068400029692A692B690FD0020E01011A6F1B6B8F
:10685000D9CFE9FFDACFEAFF260EE16E010EE26E34
:10686000060EFAEC02F008C21CF109C21DF10AC2C0
:106870001EF10BC21FF10CC220F10DC221F104C2A6
:1068800022F105C223F106C224F107C225F10EC28E
:1068900000F000EE06F0D950E926DA50EA22EF5077
:1068A00001012219016E005001140009D8B401D071
:1068B00011D00FC200F000EE07F0D950E926DA50EF
:1068C000EA22EF502319016E005001140009D8B4D8
:1068D00002D000D013D000D010C200F000EE08F0BB
:1068E000D950E926DA50EA22EF5001012419016E4D
:1068F000005001140009D8B402D000D013D000D049
:1069000011C200F000EE09F0D950E926DA50EA226F
:10691000EF5001012519016E005001140009D8B48F
:1069200002D000D002D000D009D012C22CF113C284
:106930002DF114C22EF115C22FF10ED000EE06F08B
:10694000D950E926DA50EA22EECF2CF1EECF2DF124
:10695000EECF2EF1EECF2FF10101140E316F010EAB
:10696000326F1CD80101260EC36F010EC46F060ED4
:10697000C56F1C0EC66FC76B43EC28F00101140EE7
:10698000CB6F010ECC6F1C0ECD6FCE6B6BEC26F077
:10699000A9EC28F01200FFFF38D73101FFFF43D0E8
:1069A00031C1E9FF32C1EAFFEECFC5F1EDCFC6F14B
:1069B000D3EC39F031C1E9FF32C1EAFF00C0EEFF8C
:1069C00001C0EDFF010100EE02F03151E926325124
:1069D000EA22EECFC5F1EDCFC6F1D3EC39F00101DB
:1069E00000EE02F03151E9263251EA2200C0EEFFFA
:1069F00001C0EDFF00EE06F03151E9263251EA22E6
:106A0000EECFC5F1EDCFC6F1D3EC39F0010100EEC8
:106A100006F03151E9263251EA2200C0EEFF01C0F2
:106A2000EDFF1200FFFFBCD7FFFF0BD00501AD6BE0
:106A30000501AC6B0B0E4FEC00F0010E00D0120004
:106A4000FFFFF4D76601FFFF99D0ACC500F000A0AE
:106A500001D001D003D0006A016A8ED0200E01015E
:106A6000696F6A6B66C1E9FF67C1EAFFEF50D8A49E
:106A700001D001D005D0FF0E006EFF0E016E7CD05C
:106A800066C17AF167C17BF1AAEC3AF000C066F109
:106A900001C067F16BD069C17AF16AC17BF1010174
:106AA0006B0E7C6F010E7D6F0F0E7E6FA00E72EC71
:106AB00001F001016B51D8A401D001D038D066C1DA
:106AC0007AF167C17BF17FEC3EF000500101686F05
:106AD0000C0E686501D001D002D00C0E686F66C143
:106AE0007AF167C17BF101016E0E7C6F010E7D6F43
:106AF00068517E6F7F6BD2EC3CF001500010D8A43F
:106B000001D001D00ED06CC161F26DC162F20501FD
:106B1000010EAD2701EE6CF0EECF00F0EDCF01F0ED
:106B20002BD00F0E01016927000E6A231FD001012F
:106B30006B51040AD8A401D001D013D001EE6CF03F
:106B4000EE52ED50FF0AFF0ED8B4EF18D8B401D0C2
:106B500001D005D06CC169F16DC16AF101D007D0D7
:106B600005D0FF0E006EFF0E016E06D094D7FF0E0B
:106B7000006EFF0E016E00D01200FFFF66D7FFFF10
:106B80000FD00501AB6B0501AC910501AD53D8B435
:106B900001D001D003D00501010EAD5F1200FFFF4F
:106BA000F0D76A01FFFF17D06AC163F26BC164F2CC
:106BB0006AC181F16BC182F1A00EC8EC00F0006ED9
:106BC00000C002F0036A03500210000ED8B4010E98
:106BD00000D01200FFFFE8D7FFFF2BD057EC01F0E9
:106BE00001016A6F0201010E6327000E6423010197
:106BF0006A51030AD8A401D001D00AD057EC01F0A1
:106C000001016A6F0201010E6327000E64230CD09C
:106C100001016A51040AD8A401D001D005D0FF0EA9
:106C2000E8CF63F2E8CF64F201016A5100D01200AC
:106C3000FFFFD4D7FFFF09D063EC01F063C200F07F
:106C400064C201F000D01200FFFFF6D7FFFF08D0AA
:106C50000501AC81200E006E016A00D01200FFFF1A
:106C6000F7D7AD01FFFF1CD0ADC163F2AEC164F236
:106C7000ADC1ABF505013F0EAB17ADC1AFF1AEC174
:106C8000B0F1A00E61EC00F0006E00C002F0036AEB
:106C900003500210000ED8B4010E00D01200FFFF06
:106CA000E3D7FFFF27D00101AD6F0101AD5110EC1B
:106CB00001F00009D8B401D001D002D0000E18D0E4
:106CC0000501010EAB270201010E6327000E6423AC
:106CD0003F0E0501AB6501D001D008D00CD863C2CE
:106CE000AFF164C2B0F1A00E61EC00F0010E00D073
:106CF0001200FFFFD8D7FFFF14D00501AB6B41ECAA
:106D000001F000D0A00EB1EC01F00009D8A401D030
:106D100001D0F8D763C200F064C201F000D01200C5
:106D2000FFFFEBD70001FFFF22D061C26AF162C210
:106D30006BF138DF0101006B016B01D04DDF010108
:106D40000051006E0151016E004B012B01510118E1
:106D500002E100510018D8A401D001D0EFD76ADFBA
:106D600063C200F064C201F000D01200FFFFDDD763
:106D70000601FFFFD8D001012B0E406F010E416FBD
:106D8000140E426F436BDEEC26F001012B51F00B29
:106D9000400AD8B401D001D001D0BFD02BC100F03F
:106DA0000F0E0016D8900036D8900034EC0F010179
:106DB0000E6F140E0E6501D001D001D0AED00101CE
:106DC0000E51D8B401D001D009D0170E406F010E7A
:106DD000416F0E51426F436BDEEC26F035C111F16D
:106DE00036C112F10101356B366B2B0EC36F010EEC
:106DF000C46F140EC56FC66B34EC3AF0001C026E03
:106E0000011C036E02C013F103C014F101010E5105
:106E1000D8B401D001D012D0170EC36F010EC46FC9
:106E20000E51C56FC66B34EC3AF0001C026E011CAB
:106E3000036E02C015F103C016F103D00101156BFA
:106E4000166B0101130EC36F010EC46F040EC56FE4
:106E5000C66B34EC3AF000C00FF101C010F1010133
:106E60002B0EC36F010EC46FC8D801011051121947
:106E700002E10F511119D8B401D006D02B51F00BFB
:106E8000400AD8B402D000D002D000D001D045D002
:106E900006C1E1FF07C1E2FFE250E110D8B401D022
:106EA00001D00CD0E1CFE9FFE2CFEAFF3BC1EEFF1A
:106EB0003CC1EEFF3DC1EEFF3EC1EEFF010100EE21
:106EC00006F00851E9260951EA2237C1EEFF38C120
:106ED000EEFF39C1EEFF3AC1EEFF0AC1E9FF0BC177
:106EE000EAFF34C1EFFF0E5101EE2DF0EECF00F0BE
:106EF000EDCF01F0005E000E015AEC0E0024006E92
:106F0000FF0E0120016E0CC1E9FF0DC1EAFF00C0B8
:106F1000EEFF01C0EDFF010E04D03EEC27F0000EA5
:106F200000D01200FFFF27D7AA01FFFF64D0450E53
:106F30000101AF6FB06B140EAD25B16F000EAE2125
:106F4000B26F0201010E6927000E6A2301EEB3F051
:106F500069C2EEFF6AC2EDFF0101B56BB66B640E4C
:106F6000B76FAC51B86FB96BBA6B04C2BBF105C255
:106F7000BCF106C2BDF107C2BEF100EE06F0AA5197
:106F8000E926AB51EA22EECFBFF1EECFC0F1EECF52
:106F9000C1F1EECFC2F1AF0EC36F010EC46F2DD899
:106FA0000101AF0EC36F010EC46F140EC56FC66B27
:106FB00034EC3AF000C0B9F101C0BAF1AAC1C3F192
:106FC000ABC1C4F10101C56B140EAD25C66F000E37
:106FD000AE21C76F43EC28F00101AF0ECB6F010E5D
:106FE000CC6F140ECD6FCE6B6BEC26F0006A016A8D
:106FF00000D01200FFFF9BD7C301FFFF48D0010163
:1070000000EE02F0C351E926C451EA22EECFC5F1E9
:10701000EDCFC6F1D3EC39F0010100EE02F0C3511F
:10702000E926C451EA2200C0EEFF01C0EDFF00EEE8
:1070300004F0C351E926C451EA22EECFC5F1EDCFE9
:10704000C6F1D3EC39F0010100EE04F0C351E9269A
:10705000C451EA2200C0EEFF01C0EDFF00EE0AF0CD
:10706000C351E926C451EA22EECFC5F1EDCFC6F1F6
:10707000D3EC39F0010100EE0AF0C351E926C45106
:10708000EA2200C0EEFF01C0EDFF1200FFFFB7D7FC
:10709000FFFF0ED00501AE6B0501AF8184EC25F03A
:1070A00019EC1FF006EC2DF092EC05F01200FFFF3A
:1070B000F1D7FFFF76D1010E0101006F5ED1010112
:1070C000006B42D101014D0E066F020E076F010EDB
:1070D000086F010E096F8CEC27F0006E00C002F003
:1070E000036A03500210D8A401D001D001D045D1C9
:1070F000010E0101006F0151D8A401D001D004D0CC
:10710000020EE8CFAEF50DD001010151060AD8A458
:1071100001D001D004D0050EE8CFAEF502D03EEC90
:1071200027F02BD10101006B32EC1FF00009D8B41D
:1071300001D001D002D00501AE6B1FD10101020EBA
:10714000066F010E076F4D0E086F020E096F010EDC
:107150000A6F010E0B6F470E0C6F020E0D6FB9EC2C
:1071600036F0006E00C002F0036A03500210D8B47B
:1071700001D001D046D0010E0101006F0105D8A455
:1071800001D001D021D0030EE8CFAEF5AFC500F09D
:1071900000A001D001D017D00229D8B40329D8B457
:1071A0000429D8B40529D8B401D001D00CD00501E8
:1071B000AF9102C104F203C105F204C106F205C198
:1071C00007F278EC1CF01CD001010151060AD8A48A
:1071D00001D001D004D0060EE8CFAEF511D00101E8
:1071E0000151110AD8A401D001D004D0070EE8CF74
:1071F000AEF506D00101006B3EEC27F00501AE6B49
:1072000004D03EEC27F00501AE6BB7D001014D0E66
:10721000066F020E076F01EE08F047C2EEFF48C28C
:10722000EDFF50EC2FF0006E00C002F0036A035037
:107230000210D8B401D001D002D00501AE6B01011B
:10724000006B9BD001014D0E066F020E076F01EE21
:1072500008F047C2EEFF48C2EDFFD1EC0BF0006E24
:1072600000C002F0036A03500210D8B401D001D06C
:1072700002D00501AE6B0101006B7FD00501AE6B42
:107280000201000E485D2A0ED8B4475DD8B001D087
:1072900001D033D00101010E066F010E076FB00E51
:1072A000086F050E096F470E0A6F020E0B6F490E2D
:1072B0000C6F020E0D6F4B0E0E6F020E0F6F04EC73
:1072C0003BF0006E00C002F0036A03500210D8B415
:1072D00001D001D010D001010151080AD8A401D079
:1072E00001D006D0010E006F040EE8CFAEF502D03B
:1072F0000501AE6B02D00501AE6B3EEC27F03DD030
:1073000044EC26F00009D8B401D001D01CD0010112
:107310004D0E066F020E076F086BB00E096F050E5B
:107320000A6F47C20BF101EE0CF049C2EEFF4AC2F0
:10733000EDFF01EE0EF04BC2EEFF4CC2EDFF86EC0E
:107340003BF00501AE6B19D0AEC5E8FF000A01E1C4
:10735000B9D6010A01E1B6D6030A01E1EFD6010A66
:107360008DE0070ACDE0010A01E1DCD6030A01E164
:1073700069D7010A01E14AD700D001010051D8A420
:1073800001D001D09CD644EC0AF0E2EC1AF070C5B2
:1073900000F000A001D001D002D00501AF91120091
:1073A000FFFF89D6C501FFFF12D0C5C1C7F1C6C115
:1073B000C8F10101C851D96EC751C86FD950C76F04
:1073C000C7C100F0C8C101F000D01200FFFFEDD727
:1073D000AC01FFFF47D0ACC1B0F1ADC1B1F1AEC15E
:1073E000B2F1AFC1B3F1B00ED96E010EDA6E00EE9C
:1073F00003F0D950E926DA50EA22EF50E16E00EEB0
:1074000003F0D950E926DA50EA22DFCFEFFFE1CFCF
:10741000DFFF00EE02F0D950E926DA50EA22EF5001
:10742000F36E10EE01F0D950E126DA50E22200EEC0
:1074300002F0D950E926DA50EA22E7CFEFFF00EE5A
:1074400001F0D950E926DA50EA22F3CFEFFFB0C1BC
:1074500000F0B1C101F0B2C102F0B3C103F000D03D
:107460001200FFFFB8D7C301FFFF72D00101CB6B41
:10747000CC6BCD6BCE6BD890C631F46EC531F36E4C
:10748000C3C1E1FFC4C1E2FF17D0E1CFE9FFE2CF02
:10749000EAFF020EE126000EE222EECF00F0EDCF71
:1074A00001F0026A036A01010050CB270150CC238E
:1074B0000250CD230350CE23F350006EF450016EE2
:1074C000010EF35E000EF45A01500010D8A401D052
:1074D00001D0DBD70101C5A101D001D009D0E7500F
:1074E000CB27010ED8B0CC27D8B0CD27D8B0CE2727
:1074F000CBC1C7F1CCC1C8F1CDC1C9F1CEC1CAF170
:1075000015D00101CD6BCE6BCB51F324CB6FCC5199
:10751000F420CC6FCD6BD8B0CD2BCE6BCBC1C7F1E7
:10752000CCC1C8F1CDC1C9F1CEC1CAF1C9C1F3FF07
:10753000CAC1F4FFF450F310D8A401D001D0E1D7B0
:107540000101CB1D006ECC1D016E00D01200FFFFAB
:107550008DD77A01FFFF21D07AC1E1FF7BC1E2FF25
:107560000ED0600ED96406D000D07B0ED96002D058
:1075700000D002D000D002D0E00EE726E652E7505D
:10758000D96ED950D8A401D001D0EBD77AC100F080
:107590007BC101F000D01200FFFFDED77601FFFFB4
:1075A00031D078C1F3FF79C1F4FF76C1D9FF77C13B
:1075B000DAFF1AD0F3CFF6FFF4CFF7FF010EF32670
:1075C000000EF422D9CFE9FFDACFEAFFD94ADA2A4E
:1075D000050EF76403D00800F55005D0F6CFE1FFA3
:1075E000F7CFE2FFE750EF6E01017A077A29D8A4BE
:1075F00001D001D0DFD776C100F077C101F000D013
:107600001200FFFFCED70601FFFF7ED00101180E4A
:10761000406F010E416F080E426F436BDEEC26F0A7
:107620001AC112F11BC113F101011A6B1B6B180E69
:10763000C36F010EC46F080EC56FC66B34EC3AF011
:10764000001C026E011C036E02C014F103C015F190
:107650000AC1E1FF0BC1E2FFF80EE72608C140F1C5
:1076600009C141F1E7500101426F436BDEEC26F0A6
:1076700008C1C3F109C1C4F10AC1E9FF0BC1EAFFA6
:10768000EF500101C56FC66B34EC3AF0001C026E7E
:10769000011C036E02C016F103C017F10101140EA4
:1076A000C36F010EC46F040EC56FC66B34EC3AF0A5
:1076B00000C010F101C011F10101180E406F010E60
:1076C000416F7AD806C1E9FF07C1EAFF18C1EFFF91
:1076D0000CC1E9FF0DC1EAFF1CC1EEFF1DC1EDFFAA
:1076E0000EC1E9FF0FC1EAFF1EC1EEFF1FC1EDFF92
:1076F00001011351111902E112511019000ED8B4F1
:10770000010E00D01200FFFF81D70601FFFF52D00B
:107710000101116B0851106F126B136B0CC114F146
:107720000DC115F10EC116F10FC117F1180E466FFC
:10773000010E476F09C148F10AC149F10B514A6F67
:107740004B6BE5EC3DF00101100E406F010E416FF7
:1077500033D80101100EC36F010EC46F080E0B2544
:10776000C56FC66B000EC62334EC3AF000C012F1B0
:1077700001C013F106C1AAF107C1ABF1010E01016D
:10778000AC6F080E0B25AD6FAE6B000EAE2395EC03
:1077900037F00101100ECB6F010ECC6F080E0B25D8
:1077A000CD6FCE6B000ECE236BEC26F0A9EC28F04B
:1077B0001200FFFFADD74001FFFF48D0010100EEEE
:1077C00004F04051E9264151EA22EECFC5F1EDCF58
:1077D000C6F1D3EC39F0010100EE04F04051E92686
:1077E0004151EA2200C0EEFF01C0EDFF00EE06F0BD
:1077F0004051E9264151EA22EECFC5F1EDCFC6F165
:10780000D3EC39F0010100EE06F04051E926415178
:10781000EA2200C0EEFF01C0EDFF00EE02F0405191
:10782000E9264151EA22EECFC5F1EDCFC6F1D3EC06
:1078300039F0010100EE02F04051E9264151EA22FF
:1078400000C0EEFF01C0EDFF1200FFFFB7D7260119
:10785000FFFF04D00101262B000E272326C1F6FFCF
:1078600027C1F7FF050EF76404D00800FFFFF550AD
:1078700005D0F6CFE9FFF7CFEAFFEF50200AD8B4E2
:10788000E9D726C1F6FF27C1F7FF050EF76404D03C
:107890000800FFFFF55005D0F6CFE9FFF7CFEAFF6C
:1078A000EF50090A0101D8B4D6D7296B2A6B286B8F
:1078B00026C1F6FF27C1F7FF050EF76404D00800C4
:1078C000FFFFF55005D0F6CFE9FFF7CFEAFFEF5005
:1078D0002D0AD8A403D0010E282B15D026C1F6FFFF
:1078E00027C1F7FF050EF76404D00800FFFFF5502D
:1078F00005D0F6CFE9FFF7CFEAFFEF502B0AD8A467
:1079000005D0010E01012627000E272326C1F6FF10
:1079100027C1F7FF050EF76404D00800FFFFF550FC
:1079200005D0F6CFE9FFF7CFEAFFEF50EAEC02F01F
:10793000D8A027D00A0E026E036A29C100F02AC11E
:1079400001F0EAEC1FF026C1F6FF27C1F7FF050E94
:10795000F76404D00800FFFFF55005D0F6CFE9FF2B
:10796000F7CFEAFFEF500424006E000E0520016EF1
:10797000D00E00240101296FFF0E01202A6F010E95
:10798000C2D70101285129C100F02AC101F0D8B4A1
:1079900005D0001E011E002AD8B4012A1200FFFFE4
:1079A00058D77A01FFFF01017E51006E7F51016EB1
:1079B0007E07000E7F5B01500010D8B464D07AC1FE
:1079C000F6FF7BC1F7FF050EF76404D00800FFFF48
:1079D000F55005D0F6CFE9FFF7CFEAFFEF500009E9
:1079E000D8B424D07CC1F6FF7DC1F7FF050EF76443
:1079F00004D00800FFFFF55005D0F6CFE9FFF7CF20
:107A0000EAFFEF50006E7AC1F6FF7BC1F7FF050E6B
:107A1000F76404D00800FFFFF55005D0F6CFE9FF6A
:107A2000F7CFEAFFEF500018D8B426D07AC1F6FF9E
:107A30007BC1F7FF050EF76404D00800FFFFF55087
:107A400005D0F6CFE9FFF7CFEAFFEF50006E016AED
:107A50007CC1F6FF7DC1F7FF050EF76404D0080076
:107A6000FFFFF55005D0F6CFE9FFF7CFEAFFEF5063
:107A7000005E000E015A09D001017A2B000E7B2313
:107A80007C2B7D2390D7006A016A1200FFFF8BD701
:107A90007601FFFF76C102F077C103F078C1F3FFF2
:107AA00079C1F4FF01017A51006E7B51016E7A07B2
:107AB000000E7B5B01500010D8B43CD0F3CFF6FF32
:107AC000F4CFF7FFF32A000EF422050EF76404D07A
:107AD0000800FFFFF55005D0F6CFE9FFF7CFEAFF2A
:107AE000EF50016E02C0F6FF03C0F7FF022A000E3E
:107AF0000322050EF76404D00800FFFFF55005D0FF
:107B0000F6CFE9FFF7CFEAFFEF50006E0150005CBF
:107B100001017C6F7D6BD8A07D0700BE7D0701BE93
:107B20007D2B7D517C11D8B4BDD77CC100F07DC1C7
:107B300001F002D0006A016A1200FFFFABD7070113
:107B4000FFFF07C1D9FF08C1DAFF01010C510B117A
:107B5000D8B420D00B07D8A00C0709C1F6FF0AC182
:107B6000F7FF092B000E0A23D9CFE9FFDACFEAFF8E
:107B7000D94ADA2A050EF76403D00800F55005D07B
:107B8000F6CFE1FFF7CFE2FFE750EF6EEF50D8A45A
:107B9000DCD701010B51006E0C51016E0B07000E7A
:107BA0000C5B01500010D8B408D0D9CFE9FFDACF70
:107BB000EAFFD94ADA2AEF6AECD707C100F008C118
:107BC00001F01200FFFFBDD74601FFFF48C1F3FFE0
:107BD00049C1F4FF46C1D9FF47C1DAFF01014A514B
:107BE000006E4B51016E4A07000E4B5B01500010B6
:107BF000D8B41AD0F3CFF6FFF4CFF7FFF32A000E74
:107C0000F422D9CFE9FFDACFEAFFD94ADA2A050E02
:107C1000F76403D00800F55005D0F6CFE1FFF7CFA9
:107C2000E2FFE750EF6EDAD746C100F047C101F03E
:107C30001200FFFFCBD7FFFF066AFFFF046A056A49
:107C40000250031003E1006A016A000C1F0E0612C5
:107C5000D890062A02360336FCE303320232025081
:107C6000005C0350015804E3016E0250005ED880AE
:107C700004360536062E06BAF0D706AE05D0041E29
:107C8000042AD8B40506051E0450026E0550036E82
:107C900006AC000C001E002AD8B40106011E000C20
:107CA000FFFF0AD03C0ED66ED768070ED56ED58E74
:107CB000F284F28A1200FFFFF5D7FFFF0BD065C2F6
:107CC00000F066C201F067C202F068C203F000D0A3
:107CD0001200FFFFF4D7FFFF10D0F2A401D001D0B3
:107CE0000AD0D7683C0ED66E0201652B000E6623C3
:107CF00067236823F2941200FFFFEFD77A01FFFF9A
:107D00007AC1F3FF7BC1F4FFF3CFF6FFF4CFF7FFA7
:107D1000F32A000EF422050EF76404D00800FFFFDA
:107D2000F55005D0F6CFE9FFF7CFEAFFEF50000995
:107D3000D8A4EAD7F3CF00F0F4CF01F001017A51D3
:107D4000005E7B51015AFF0E0024006EFF0E0120E1
:107D5000016E1200FFFFD4D7FFFF1AD0E96E10D0DA
:107D6000040EE16E07D0500ED96E00D001D000D0C5
:107D7000D92EFDD7E106E128D8A401D001D0F3D750
:107D8000E906E928D8A401D001D0EAD71200FFFF04
:107D9000E5D7FFFFEFCF00F0EE2AEFCF01F0000EA6
:107DA000EE22EFCF02F0EE22EFCF03F0EE22120030
:107DB0000900F5CFEEFFFFFFEA50E262F9D7E95084
:107DC000E162F6D71200EE6AFFFFEA50E262FBD7EB
:087DD000E950E162F8D712004E
:020000040030CA
:04000000FFFAFCFE09
:020000040000FA
:00000001FF
